:020000040000FA
:06000000B2EF3EF0120019
:06080000B2EF3EF0120011
:06082A0006003C7E000008
:10083000E90100000C0000003B7E0000B502000052
:1008400001000000357E0000FA00000006000000F4
:10085000BD7D0000B402000001000000287E000001
:10086000DC0100000D000000247E0000AA02000050
:040870000400000080
:0C08740004001200D9CFE6FFE1CFD9FF4D
:1008800081E945E8030E056E0101E551010A17E013
:10089000010A2AE10A0EE45D09E10001DA51016E64
:1008A000DB51026EDC51036EDD511DD0020100519F
:1008B000016E0151026E0251036E035114D00A0EF3
:1008C000E45D09E10001DE51016EDF51026EE0518D
:1008D000036EE15108D002010451016E0551026E10
:1008E0000651036E0751046E97EC0AF0030A2DE0DF
:1008F000070A1BE0010A0AE0050A04E0010A02E017
:10090000030A35E10D0EE66E730E34D0080EE66E66
:10091000730E0DEC0AF00001CB51E66EE66A030E91
:10092000E66ECF0EE66E000E2CD0030EE66E730E52
:100930000DEC0AF0DCC1E6FFDDC1E6FFDEC1E6FF3B
:10094000DFC1E6FF9BEC0AF017D0FE0EE66E720EDA
:100950000DEC0AF0E0C1E6FFE1C1E6FFE2C1E6FF0F
:10096000E3C1E6FF9BEC0AF0040E056E05D0F90E1C
:10097000E66E720E0DEC0AF00101E55106E160EC45
:100980000AF0E66E5DEC36F005D060EC0AF0E66E3B
:1009900096EC36F045E946E9E7CFD9FF1200D9CF0A
:1009A000E6FFE1CFD9FF81E958E8136A146A156AB6
:1009B000166A176A186AE70E926ED00E936EB80E1A
:1009C000946EF19E8A86D0B604D0E66A00EC2FF0D1
:1009D00041E9170EE66E9BEC3DF041E959EC0AF057
:1009E000750EE66E60EC3DF041E990EC0AF0010115
:1009F000E451FF0A02E175EF09F0F40A01E16AD35C
:100A0000010A01E1C4D2030A01E12DD2010A01E188
:100A100017D20F0A01E1FED1010A01E1D5D1030A83
:100A200001E1BFD1010A01E1AAD1070A01E1A2D186
:100A3000010A01E196D1030A01E187D1010A02E02E
:100A400083EF09F0020EF66E770EF76E0900F5CF10
:100A500060F00900F5CF61F00900F5CF62F0090000
:100A6000F5CF63F00900F5CF64F00900F5CF65F02C
:100A70000900F5CF66F00900F5CF67F00900F5CF62
:100A800068F00900F5CF69F00900F5CF6AF00900B8
:100A9000F5CF6BF00900F5CF6CF00900F5CF6DF0E4
:100AA0000900F5CF6EF00900F5CF6FF00900F5CF22
:100AB00070F00900F5CF71F00900F5CF72F0090070
:100AC000F5CF73F00900F5CF74F00900F5CF75F09C
:100AD0000900F5CF76F00900F5CF77F00900F5CFE2
:100AE00078F00900F5CF79F00900F5CF7AF0090028
:100AF000F5CF7BF00900F5CF7CF00900F5CF7DF054
:100B00000900F5CF7EF00900F5CF7FF00900F5CFA1
:100B100080F00900F5CF81F00900F5CF82F00900DF
:100B2000F5CF83F00900F5CF84F00900F5CF85F00B
:100B30000900F5CF86F00900F5CF87F00900F5CF61
:100B400088F00900F5CF89F00900F5CF8AF0090097
:100B5000F5CF8BF00900F5CF8CF00900F5CF8DF0C3
:100B60000900F5CF8EF00900F5CF8FF00900F5CF21
:100B700090F00900F5CF91F00900F5CF92F009004F
:100B8000F5CF93F00900F5CF94F00900F5CF95F07B
:100B90000900F5CF96F00900F5CF97F00900F5CFE1
:100BA00098F00900F5CF99F00900F5CF9AF0090007
:100BB000F5CF9BF00900F5CF9CF00900F5CF9DF033
:100BC0000900F5CF9EF00900F5CF9FF00900F5CFA1
:100BD000A0F00900F5CFA1F00900F5CFA2F00900BF
:100BE000F5CFA3F00900F5CFA4F00900F5CFA5F0EB
:100BF0000900F5CFA6F00900F5CFA7F00900F5CF61
:100C0000A8F00900F5CFA9F00900F5CFAAF0090076
:100C1000F5CFABF00900F5CFACF00900F5CFADF0A2
:100C20000900F5CFAEF00900F5CFAFF00900F5CF20
:100C3000B0F00900F5CFB1F00900F5CFB2F009002E
:100C4000F5CFB3F00900F5CFB4F00900F5CFB5F05A
:100C50000900F5CFB6F00900F5CFB7F00900F5CFE0
:100C6000B8F00900F5CFB9F00900F5CFBAF00900E6
:100C7000F5CFBBF00900F5CFBCF00900F5CFBDF012
:100C80000900F5CFBEF00900F5CFBFF00900F5CFA0
:100C9000C0F00900F5CFC1F00900F5CFC2F009009E
:100CA000F5CFC3F00900F5CFC4F00900F5CFC5F0CA
:100CB0000900F5CFC6F00800F5CFC7F00001C7B7AF
:100CC0001CD02F0EC16F400EC06FC26FC787C79177
:100CD000C783C7953C0EC36FC46B0F0EC56FC66B41
:100CE000C789C78DC79BC78F600EE66E000EE66E84
:100CF0000AEC24F042E9680EC6DBF3EC20F0DDECF0
:100D00002DF017EC27F0F4EC11F0E3EC1CF0690E79
:100D1000F66E770EF76E0800F550080B02E1EDEC69
:100D20002DF08CEC2EF0380E946EB1EC21F081A8F1
:100D300084D00001C7A907D00101010EE46F0001B2
:100D4000C96BCA6BE0D2D4DBDED20001C8B303D0DA
:100D50000101020EE46F020E0101E55D01E0D3D254
:100D600031D00001C8B3C4DB020E0101E55D01E032
:100D7000CAD228D0C5DBC8A1C6D2010123D0E8DB86
:100D8000CCBFCD69BAEC0AF0A5DB0001C8A102D046
:100D90000101E4690101CB5101E1B5D20101050E68
:100DA000B1D2C0C0C9F0C1C0CAF0EF0EE66E720E7B
:100DB00034DB0101CB5102E10101A2DB0001C8A13A
:100DC000A2D20101E4699FD2E551020A15E0030AAB
:100DD00007E0010A1BE1BCDBCCBFCD69CBDB0AD04D
:100DE000EA0EE66E720E19DB32EC2EF0F3CFE6FF60
:100DF000F4CFE6FF6FDB0AD0E56B0001C8A306D095
:100E0000C9693F0ECA6F0101010EE86F0001C8B346
:100E10007AD276D2E551020A06E0020A02E0010A1D
:100E200003E12ADD01D0E56B0001C8A303D0010175
:100E3000080EE46F0001C8B166D20101030E62D250
:100E40007D0EE66E40EC3DF041E9000EE66EE66A8E
:100E5000EAEC3DF042E90101E56B2BDB156A166A0D
:100E60000101090EE46F63DB000A1EE0010A18E0CD
:100E7000030A12E0010A0CE0070A06E0010A18E181
:100E8000E50EE66E720E13D0E00EE66E720E0FD017
:100E9000DB0EE66E720E0BD0D60EE66E720E07D02B
:100EA000D10EE66E720E03D0CC0EE66E720EB5DA7F
:100EB0000001C8B302D00101E46902EC3EF011DB8D
:100EC00001E321D202EC3EF0ECDAEAEC3DF042E93B
:100ED000152A000E1622020EE66EE66AC5C0E6FF6F
:100EE000C6C0E6FFD8EC2CF0FE0EE350155C41E9DD
:100EF000E550165801E207D200C2DAF001C2DBF079
:100F000002C2DCF003C2DDF004C2DEF005C2DFF095
:100F100006C2E0F007C2E1F00101E56B01010351F7
:100F2000056E0451066E0551076E0651086E075195
:100F3000096E08510A6E09510B6E0A510C6E0B5165
:100F40000D6E0C510E6E0D510F6E0E51106EE66A45
:100F50000DEC28F041E9116A126AD890125004E6AB
:100F60005E0E115C010E125802E272DAF6D7C9C0A9
:100F7000E6FF0DEC28F041E903EC3FF001010A0E19
:100F8000E46F02014651176E4751186EBCD1E5510E
:100F9000030A31E0010A06E0020A02E0010A2CE13C
:100FA0006BDC2AD0C4DA000A14E01750E708030EFD
:100FB000185412E2C70EE66E720E2FDA0101E80E27
:100FC000175CCC6F030E1858CD6FCCC1E6FFE66EF0
:100FD0000BD00101E56B10D0C20EE66E720E1DDA69
:100FE00017EBE6FF18EBE6FF030EE66ECF0EE66E9C
:100FF000000EC5DA01D0E56B020E0001C8155DE1F7
:101000000101E7515AE193DA010A49E0030A3EE09F
:10101000010A38E0070A32E0010A45E1CB510C0D24
:1010200002018851F324E96E8951F420EA6E05EB40
:10103000EEFF06EBEEFF07EBEEFF08EBEEFF09EB32
:10104000EEFF0AEBEEFF0BEBEEFF0CEBEEFF0DEB12
:10105000EEFF0EEBEEFF0FEBEEFF10EBEEFF0001ED
:10106000CB2B380ECB5D1FE301010B0EE46F0001AB
:10107000CB6BCC6BDEEC25F074DA15D0D8D943EC11
:101080001FF010D0D4D9FEEC1EF00CD0D950050FB3
:10109000E66EDACFE6FF58EC1FF042E904D0C7D97C
:1010A00063EC1EF048E90001C7AD04D00101010E58
:1010B000E76F03D00101070EE46F020E0001C815AF
:1010C00001E121D10101E75101E11DD1080EE46FD9
:1010D000E76B19D10001CC51010BE66EF2EC25F063
:1010E00041E9C6D90001CC2BBD0EE66E720E95D932
:1010F0000001CC51E66EE66A020EE66ED00EE66E98
:10110000000E3DDA640E0001CC5D01E0FCD0A0C70A
:1011100060F0A1C761F0A2C762F0A3C763F0A4C7E3
:1011200064F0A5C765F0A6C766F0A7C767F0A8C7B3
:1011300068F0A9C769F0AAC76AF0ABC76BF0ACC783
:101140006CF0ADC76DF0AEC76EF0AFC76FF0B0C753
:1011500070F0B1C771F0B2C772F0B3C773F0B4C723
:1011600074F0B5C775F0B6C776F0B7C777F0B8C7F3
:1011700078F0B9C779F0BAC77AF0BBC77BF0BCC7C3
:101180007CF0BDC77DF0BEC77EF0BFC77FF0C0C793
:1011900080F0C1C781F0C2C782F0C3C783F0C4C763
:1011A00084F0C5C785F0C6C786F0C7C787F0C8C733
:1011B00088F0C9C789F0CAC78AF0CBC78BF0CCC703
:1011C0008CF0CDC78DF0CEC78EF0CFC78FF0D0C7D3
:1011D00090F0D1C791F0D2C792F0D3C793F0D4C7A3
:1011E00094F0D5C795F0D6C796F0D7C797F0D8C773
:1011F00098F0D9C799F0DAC79AF0DBC79BF0DCC743
:101200009CF0DDC79DF0DEC79EF0DFC79FF0E0C712
:10121000A0F0E1C7A1F0E2C7A2F0E3C7A3F0E4C7E2
:10122000A4F0E5C7A5F0E6C7A6F0E7C7A7F0E8C7B2
:10123000A8F0E9C7A9F0EAC7AAF0EBC7ABF0ECC782
:10124000ACF0EDC7ADF0EEC7AEF0EFC7AFF0F0C752
:10125000B0F0F1C7B1F0F2C7B2F0F3C7B3F0F4C722
:10126000B4F0F5C7B5F0F6C7B6F0F7C7B7F0F8C7F2
:10127000B8F0F9C7B9F0FAC7BAF0FBC7BBF0FCC7C2
:10128000BCF0FDC7BDF0FEC7BEF0FFC7BFF0CD513B
:10129000070BF36EF80EC715F310C76F600EF3D887
:1012A000116A126A640ED89012BE03D0115C000E4F
:1012B000125802E2CDD8F6D72BD9640ED89012BEC0
:1012C00003D0115C000E125802E2C2D8F6D720D922
:1012D000640ED89012BE03D0115C000E125802E2C8
:1012E000B7D8F6D701010A0E0DD0E8C1E6FF00EC31
:1012F0002FF041E91CD9CD6FC781C793C785CB6B50
:101300000101070EE46FC7EC15F00001C86B8150B6
:10131000100B01E0010EC82784EC2EF0000906E056
:10132000020E0001C827FCD8136A146AC7EC15F036
:101330003AEC04F0C1EC21F0C7EC15F0040E010109
:10134000E76E661902E7663502D06651E75C12E285
:10135000B80EE66E720E61D8E66A650EE66E010E94
:10136000E66E010EE66ED00EE66E000EE66EBBEC8B
:1013700036F046E9CE0EE66E000EE66E74EC28F00E
:1013800042E962EC3EF000D90001C2510101CF6B8D
:10139000C2C0CFF1CE6BF350CE5DF450CF590CE20A
:1013A0000101E52B0A0EE45D04E141D8FAEC27F0D7
:1013B00048E98CEC2EF07DD8C7EC15F032EC3EF00D
:1013C00090D822E232EC3EF06CD81AEC3EF042E9C2
:1013D000132A000E14220001C351C41115E0140E8B
:1013E000E66EE66AC3C0E6FFC4C0E6FFD8EC2CF0A8
:1013F000FE0EE350D8801354145041E9E55804E23E
:10140000E66A00EC2FF041E9C7EC15F0C9C0E6FF31
:101410000DEC28F041E9F7EF04F0E66EE66ACE0E37
:10142000E66E000EE66E8DEC34F045E91200DEC08B
:10143000E6FFDFC0E6FFE0C0E6FFE1C0E6FFDAC09E
:10144000E6FFDBC0E6FFDCC0E6FFDDC0E6FF120022
:101450008A84990EE66ECBEC3EF041E98A94990EAF
:10146000E66ECBEC3EF041E9112A000E122212008A
:1014700078D80101CC51016ECD51026ECE51036E70
:10148000CF51046E1200E66EE66A600EE66E000E44
:10149000E66E020EE66E770EE66EA5EC1DF046E9EE
:1014A000120072D80101A80ECC5F610ECD5BBAEFBD
:1014B0000AF0000EE66EE66A4AEC3EF042E91200DF
:1014C00003EBE6FF04EBE6FF05EBE6FFCE0EE66E70
:1014D000000E1200030EE66ECE0EE66E000EBFEF9B
:1014E0000AF052D80101F350A808610EF45412001A
:1014F0000101060EE46FC0C0C9F0C1C0CAF01200FD
:10150000040EE46F0001010EC96F110ECA6F1200C4
:101510001E0EE66E80EC3DF041E9116A126A12007F
:10152000000EE66EE66A1AEC3EF042E91200000197
:10153000C751070B120001EBE6FF02EBE6FF03EBDE
:10154000E6FF04EBE6FF0DEC35F048E938EF0AF072
:10155000F40EE66E720E61DFA1C2CCF10101CD6B1B
:101560001200A2C2CCF1A3C2CDF1A4C2CEF1A5C299
:10157000CFF11200CCC1E6FFCDC1E6FF1200E66E4E
:101580005DEC36F045E91200F3CFCCF1F4CFCDF1AC
:02159000120047
:0E15920003EBE6FF04EBE6FF05EBE6FF06EBDE
:1015A000E6FFEECFE6FFEECFE6FFEECFE6FFEECFB3
:1015B000E6FF19EC35F007EBE6FF08EBE6FF09EB79
:1015C000E6FF0AEBE6FF08E8EECFE6FFEECFE6FF28
:1015D000EECFE6FFEECFE6FF19EC35F02D502926D1
:1015E0002E502A222F502B2230502C2244E90BEB74
:1015F000E6FF0CEBE6FF0DEBE6FF0EEBE6FF08E87F
:10160000EECFE6FFEECFE6FFEECFE6FFEECFE6FF52
:1016100019EC35F02D5029262E502A222F502B223E
:1016200030502C2244E908E8EECFE6FFEECFE6FF8B
:10163000EECFE6FFEECFE6FF2D5029262E502A22D0
:101640002F502B2230502C2244E924E903EBE6FFF3
:1016500004EBE6FF05EBE6FF06EBE6FFEECFE6FF69
:10166000EECFE6FFEECFE6FFEECFE6FF19EC35F06A
:1016700007EBE6FF08EBE6FF09EBE6FF0AEBE6FF08
:1016800008E8EECFE6FFEECFE6FFEECFE6FFEECFC7
:10169000E6FF19EC35F031502D2632502E22335012
:1016A0002F223450302244E90BEBE6FF0CEBE6FF2F
:1016B0000DEBE6FF0EEBE6FF08E8EECFE6FFEECF20
:1016C000E6FFEECFE6FFEECFE6FF19EC35F0315046
:1016D0002D2632502E2233502F223450302244E90E
:1016E00008E8EECFE6FFEECFE6FFEECFE6FFEECF67
:1016F000E6FF31502D2632502E2233502F22345007
:10170000302244E924E903EBE6FF04EBE6FF05EBB6
:10171000E6FF06EBE6FFEECFE6FFEECFE6FFEECF0D
:10172000E6FFEECFE6FF19EC35F007EBE6FF08EB3E
:10173000E6FF09EBE6FF0AEBE6FF08E8EECFE6FF7F
:10174000EECFE6FFEECFE6FFEECFE6FF19EC35F089
:101750003550312636503222375033223850342219
:1017600044E90BEBE6FF0CEBE6FF0DEBE6FF0EEBBF
:10177000E6FF08E8EECFE6FFEECFE6FFEECFE6FFAE
:10178000EECFE6FF19EC35F03550312636503222D7
:10179000375033223850342244E908E8EECFE6FFD0
:1017A000EECFE6FFEECFE6FFEECFE6FF3550312677
:1017B00036503222375033223850342244E924E95B
:1017C000E552E5500E6EE5500D6EE5500C6EE7509B
:1017D0000B6EE552E5500A6EE550096EE550086E55
:1017E000E750076EE552E550066EE550056EE55090
:1017F000046EE750036E000CD89006BED880063207
:1018000005320432D8900ABED8800A320932083232
:10181000D8900EBED8800E320D320C32000C036A06
:10182000046AEE50056EEE50066E076A086AEE50C6
:10183000096EEE500A6E0B6A0C6AEE500D6EEE5099
:101840000E6E000C64E8D9CFE6FFDACFE6FFE1CFF9
:10185000D9FFE2CFDAFFA9E901EBE9FF02EBEAFFEA
:1018600006E8DDDFC9DFC8DF00EE60F092DE83EB63
:101870000FF084EB10F085EB11F086EB12F087EBA4
:1018800013F088EB14F089EB15F08AEB16F08BEB74
:1018900017F08CEB18F08DEB19F08EEB1AF001EBD2
:1018A000E9FF02EBEAFFBBDFA7DFA6DFA5DF00EE63
:1018B00090F06FDE03EBE6FF04EBE6FF05EBE6FFDF
:1018C00006EBE6FF03EBE6FF04EBE6FF05EBE6FFC6
:1018D00006EBE6FF19EC35F007EBE6FF08EBE6FF59
:1018E00009EBE6FF0AEBE6FF07EBE6FF08EBE6FF96
:1018F00009EBE6FF0AEBE6FF19EC35F00BEBE6FF30
:101900000CEBE6FF0DEBE6FF0EEBE6FF0BEBE6FF65
:101910000CEBE6FF0DEBE6FF0EEBE6FF19EC35F006
:1019200031502D2632502E2233502F223450302267
:1019300044E92D5029262E502A222F502B22305098
:101940002C2244E90201295038272A5039232B50F0
:101950003A232C503B23FC0EE3CFE6FFE3CFE6FF18
:10196000E3CFE6FFE3CFE6FFC4EC35F0FC0EE3CFB8
:10197000E6FFE3CFE6FFE3CFE6FFE3CFE6FF03EBCF
:10198000E6FF04EBE6FF05EBE6FF06EBE6FF19ECEE
:1019900035F0E552E550066EE550056EE550046EF3
:1019A000E750036EFC0EE3CFE6FFE3CFE6FFE3CFA5
:1019B000E6FFE3CFE6FF07EBE6FF08EBE6FF09EB08
:1019C000E6FF0AEBE6FF19EC35F0E552E5500A6E4A
:1019D000E550096EE550086EE750076EFC0EE3CF48
:1019E000E6FFE3CFE6FFE3CFE6FFE3CFE6FF0BEB57
:1019F000E6FF0CEBE6FF0DEBE6FF0EEBE6FF19EC66
:101A000035F0E552E5500E6EE5500D6EE5500C6E6A
:101A1000E7500B6E19EC35F00201295020272A50AF
:101A200021232B5022232C50232344E90FEBE6FFE4
:101A300010EBE6FF11EBE6FF12EBE6FF0FEBE6FF24
:101A400010EBE6FF11EBE6FF12EBE6FF19EC35F0C9
:101A500013EBE6FF14EBE6FF15EBE6FF16EBE6FFF4
:101A600013EBE6FF14EBE6FF15EBE6FF16EBE6FFE4
:101A700019EC35F017EBE6FF18EBE6FF19EBE6FF84
:101A80001AEBE6FF17EBE6FF18EBE6FF19EBE6FFB4
:101A90001AEBE6FF19EC35F031502D2632502E228C
:101AA00033502F223450302244E92D5029262E5015
:101AB0002A222F502B2230502C2244E90201295097
:101AC0003C272A503D232B503E232C503F23FC0E15
:101AD000E3CFE6FFE3CFE6FFE3CFE6FFE3CFE6FFAA
:101AE000C4EC35F0FC0EE3CFE6FFE3CFE6FFE3CF37
:101AF000E6FFE3CFE6FF0FEBE6FF10EBE6FF11EBAF
:101B0000E6FF12EBE6FF19EC35F0E552E550126EF8
:101B1000E550116EE550106EE7500F6EFC0EE3CFEE
:101B2000E6FFE3CFE6FFE3CFE6FFE3CFE6FF13EB0D
:101B3000E6FF14EBE6FF15EBE6FF16EBE6FF19EC0C
:101B400035F0E552E550166EE550156EE550146E11
:101B5000E750136EFC0EE3CFE6FFE3CFE6FFE3CFE3
:101B6000E6FFE3CFE6FF17EBE6FF18EBE6FF19EB26
:101B7000E6FF1AEBE6FF19EC35F0E552E5501A6E78
:101B8000E550196EE550186EE750176E19EC35F0F8
:101B90000201295024272A5025232B5026232C507C
:101BA000272344E907EBE6FF08EBE6FF09EBE6FF36
:101BB0000AEBE6FF17EBE6FF18EBE6FF19EBE6FF93
:101BC0001AEBE6FF19EC35F00BEBE6FF0CEBE6FF4A
:101BD0000DEBE6FF0EEBE6FF13EBE6FF14EBE6FF83
:101BE00015EBE6FF16EBE6FF19EC35F02D50295EFC
:101BF0002E502A5A2F502B5A30502C5A44E90BEBB6
:101C0000E6FF0CEBE6FF0DEBE6FF0EEBE6FF0FEB5E
:101C1000E6FF10EBE6FF11EBE6FF12EBE6FF19EC37
:101C200035F003EBE6FF04EBE6FF05EBE6FF06EB22
:101C3000E6FF17EBE6FF18EBE6FF19EBE6FF1AEB02
:101C4000E6FF19EC35F031502D5E32502E5A3350EC
:101C50002F5A3450305A44E903EBE6FF04EBE6FF19
:101C600005EBE6FF06EBE6FF13EBE6FF14EBE6FF02
:101C700015EBE6FF16EBE6FF19EC35F007EBE6FF98
:101C800008EBE6FF09EBE6FF0AEBE6FF0FEBE6FFEA
:101C900010EBE6FF11EBE6FF12EBE6FF19EC35F077
:101CA0003550315E3650325A3750335A3850345AE4
:101CB00044E9E552E5501A6EE550196EE550186E8C
:101CC000E750176EE552E550166EE550156EE5507B
:101CD000146EE750136EE552E550126EE550116E2A
:101CE000E550106EE7500F6E0FEBE6FF10EBE6FFCE
:101CF00011EBE6FF12EBE6FF0FEBE6FF10EBE6FF62
:101D000011EBE6FF12EBE6FF19EC35F013EBE6FF03
:101D100014EBE6FF15EBE6FF16EBE6FF13EBE6FF31
:101D200014EBE6FF15EBE6FF16EBE6FF19EC35F0DA
:101D300017EBE6FF18EBE6FF19EBE6FF1AEBE6FF01
:101D400017EBE6FF18EBE6FF19EBE6FF1AEBE6FFF1
:101D500019EC35F031502D2632502E2233502F22DF
:101D60003450302244E92D5029262E502A222F505B
:101D70002B2230502C2244E90201295040272A50BE
:101D800041232B5042232C504323FC0EE3CFE6FF8C
:101D9000E3CFE6FFE3CFE6FFE3CFE6FFC4EC35F0A9
:101DA000FC0EE3CFE6FFE3CFE6FFE3CFE6FFE3CFB2
:101DB000E6FF0FEBE6FF10EBE6FF11EBE6FF12EBA1
:101DC000E6FF19EC35F0E552E550126EE550116E64
:101DD000E550106EE7500F6EFC0EE3CFE6FFE3CF49
:101DE000E6FFE3CFE6FFE3CFE6FF13EBE6FF14EBFE
:101DF000E6FF15EBE6FF16EBE6FF19EC35F0E552D2
:101E0000E550166EE550156EE550146EE750136EF2
:101E1000FC0EE3CFE6FFE3CFE6FFE3CFE6FFE3CF41
:101E2000E6FF17EBE6FF18EBE6FF19EBE6FF1AEB10
:101E3000E6FF19EC35F0E552E5501A6EE550196EE3
:101E4000E550186EE750176E19EC35F00201295075
:101E500028272A5029232B502A232C502B2344E9AE
:101E6000100E0060B4D113EBE6FF14EBE6FF15EBA8
:101E7000E6FF16EBE6FF0BEBE6FF0CEBE6FF0DEBE8
:101E8000E6FF0EEBE6FF19EC35F017EBE6FF18EB7B
:101E9000E6FF19EBE6FF1AEBE6FF07EBE6FF08EBC0
:101EA000E6FF09EBE6FF0AEBE6FF19EC35F02D50F3
:101EB000295E2E502A5A2F502B5A30502C5A44E962
:101EC00017EBE6FF18EBE6FF19EBE6FF1AEBE6FF70
:101ED00003EBE6FF04EBE6FF05EBE6FF06EBE6FFB0
:101EE00019EC35F00FEBE6FF10EBE6FF11EBE6FF28
:101EF00012EBE6FF0BEBE6FF0CEBE6FF0DEBE6FF6C
:101F00000EEBE6FF19EC35F031502D5E32502E5AB3
:101F100033502F5A3450305A44E90FEBE6FF10EBA0
:101F2000E6FF11EBE6FF12EBE6FF07EBE6FF08EB3F
:101F3000E6FF09EBE6FF0AEBE6FF19EC35F013EBE1
:101F4000E6FF14EBE6FF15EBE6FF16EBE6FF03EB0F
:101F5000E6FF04EBE6FF05EBE6FF06EBE6FF19EC18
:101F600035F03550315E3650325A3750335A38508A
:101F7000345A44E9E552E550266EE550256EE550A9
:101F8000246EE750236EE552E550226EE550216E37
:101F9000E550206EE7501F6EE552E5501E6EE5508D
:101FA0001D6EE5501C6EE7501B6E1BEBE6FF1CEB35
:101FB000E6FF1DEBE6FF1EEBE6FF1BEBE6FF1CEB6F
:101FC000E6FF1DEBE6FF1EEBE6FF19EC35F01FEB1D
:101FD000E6FF20EBE6FF21EBE6FF22EBE6FF1FEB3F
:101FE000E6FF20EBE6FF21EBE6FF22EBE6FF19EC34
:101FF00035F023EBE6FF24EBE6FF25EBE6FF26EBCF
:10200000E6FF23EBE6FF24EBE6FF25EBE6FF26EBFE
:10201000E6FF19EC35F031502D2632502E22335088
:102020002F223450302244E92D5029262E502A22C6
:102030002F502B2230502C2244E9C4EC35F0FC0EFA
:10204000E3CFE6FFE3CFE6FFE3CFE6FFE3CFE6FF34
:102050001BEBE6FF1CEBE6FF1DEBE6FF1EEBE6FFCE
:1020600019EC35F0E552E5501E6EE5501D6EE55059
:102070001C6EE7501B6EFC0EE3CFE6FFE3CFE6FFDE
:10208000E3CFE6FFE3CFE6FF1FEBE6FF20EBE6FF43
:1020900021EBE6FF22EBE6FF19EC35F0E552E550C7
:1020A000226EE550216EE550206EE7501F6EFC0E4B
:1020B000E3CFE6FFE3CFE6FFE3CFE6FFE3CFE6FFC4
:1020C00023EBE6FF24EBE6FF25EBE6FF26EBE6FF3E
:1020D00019EC35F0E552E550266EE550256EE550D9
:1020E000246EE750236E44E91BEBE6FF1CEBE6FF92
:1020F0001DEBE6FF1EEBE6FF1BEBE6FF1CEBE6FF2E
:102100001DEBE6FF1EEBE6FF02012D5014272E50BB
:1021100015232F5016233050172319EC35F0295072
:102120002C272A502D232B502E232C502F2344E9CB
:102130000FEBE6FF10EBE6FF11EBE6FF12EBE6FF1D
:102140000FEBE6FF10EBE6FF11EBE6FF12EBE6FF0D
:102150002D5018272E5019232F501A2330501B238F
:1021600019EC35F0295030272A5031232B503223D7
:102170002C50332344E903EBE6FF04EBE6FF05EBC9
:10218000E6FF06EBE6FF03EBE6FF04EBE6FF05EBFD
:10219000E6FF06EBE6FF2D501C272E501D232F5087
:1021A0001E2330501F2319EC35F0295034272A50B4
:1021B00035232B5036232C50372344E9020107EBFB
:1021C00008F208EB09F209EB0AF20AEB0BF2E5520E
:0E21D000E5CFDAFFE7CFD9FF64E9000C000C81
:0221DE00F3EC20
:1021E00016F031E021EC16F0D00F056E055009080D
:1021F00002E2070E055E05500F0802E2200E055EA2
:1022000005500F0815E30228E96E000E0320EA6E60
:10221000EF50D00F066E0650090802E2070E065E68
:1022200006500F0802E2200E065E06500F0802E27A
:10223000FF0E0AD00538F00B0624E66E3FEC16F0D0
:10224000E552E750EF6E000E89EF16F0F3EC16F052
:1022500024E044EC16F0C3DF44E900090BE1D95057
:10226000060FE4EC16F0020E4CEC16F0B8DF44E971
:10227000000902E0FF0E12D005500101CF6BCF6FB5
:10228000CE6B0650CE25CC6F000ECF21CD6F3FEC2C
:1022900016F0CCC1EEFFCDC1EDFF000E89EF16F0B8
:1022A0002EEC16F085E944E821EC16F048E044EC09
:1022B00016F0CCDF44E900090BE1D950070FE4EC3C
:1022C00016F0040E4CEC16F0C1DF44E9000902E000
:1022D000FF0E36D0E66A010EE66EE66AE66AE66A48
:1022E000E66EE66AE66A05EBE6FF06EBE6FFE66AFF
:1022F000E66A0CEC2DF00CEC2DF0E552E5CFCFF1B9
:10230000E5CFCEF1E5CFCDF1E7CFCCF107EBD0F1C2
:1023100008EBD1F10101D26BD36BD051CC27D15155
:10232000CD23D251CE23D351CF233FEC16F0CCC1D5
:10233000EEFFCDC1EEFFCEC1EEFFCFC1EEFF000E2E
:1023400045E9E7CFD9FF12002EEC16F085E921EC24
:1023500016F010E021EC16F0300804E13FEC16F026
:10236000EF6A08D021EC16F0310806E13FEC16F0D8
:10237000010EEF6E000E01D0FF0E41E9E7CFD9FF4D
:1023800012002EEC16F081E942E8670E016E010E94
:10239000026E82EC16F00101CF6BCEBFCF69CEC1C9
:1023A000E6FFCFC1E6FFB5EC3BF056EC16F004E0DB
:1023B000012A000E0222EDD782EC16F0CF6BCEBFC1
:1023C000CF69CEC1E6FFCFC1E6FFD3EC3BF056ECC0
:1023D00016F004E0012A000E0222EED701EBF3FF13
:1023E00002EBF4FF89EF16F0140E6F6E0201A66B7C
:1023F0000201A76B0201A86B33EC16F0DBEC16F0C0
:102400000101876BC86BCB6BC96BCA6B12001F0EC7
:102410000101D8808755E66E87C1CCF10101CD6BF3
:10242000CCBFCD69670ECC27010EE8EC16F0A6EC08
:1024300031F043E912000001E35106E1DBDBD7ECA8
:1024400031F042E90201B46B1200FF0012002EECE1
:1024500016F081E963E80168DBEC16F001016751D1
:10246000510A01E1F8D1010A01E1E8D1020A01E1D2
:1024700088D1010A01E153D1100A01E132D1040AE5
:1024800001E1D7D0110A0EE01E0A01E02AD3016A49
:10249000B30EE66E720EFDEC16F045E90101010E79
:1024A000CB6F1FD36851520A01E1B3D01F0A01E17B
:1024B0008ED00F0A01E17AD00A0A6DE00E0A60E0C0
:1024C000090A53E01C0A42E0030A31E0040A26E04C
:1024D000100A13E0080A01E004D3C00EE66E000EF5
:1024E0009DDBC00EE66E000EE66E010EC8EC16F027
:1024F000C0C0E6FF0DEC28F00FD0C10EE66E000E56
:102500008DDBC10EE66E000EE66E010EC8EC16F015
:10251000C1C0E6FFF5EC28F041E9E3D2C20EE66E59
:10252000000E7CDBC20EE66E000EE66E70D0B4ECE0
:1025300016F001E1051C04E004EBC3F005EBC4F068
:10254000010EE66EC30EE66E000E70D0B4EC16F00F
:1025500001E1051C04E004EBC5F005EBC6F0010E3B
:10256000E66EC50EE66E000E61D0E7DB05E00250B8
:102570000001C799E8B0C7890001C7B921D023D0AD
:10258000DCDB05E002500001C79BE8B0C78B00010F
:10259000C7AB19D015D0D1DB05E002500001C79DB3
:1025A000E8B0C78D0001C7AD0ED00AD0C6DB05E08C
:1025B00002500001C79FE8B0C78F0001C7AF03D02A
:1025C0000101310E02D00101300E886F8AD20268FB
:1025D000D950020F0CDB03DE44E9016EFF0E025CF2
:1025E0000BE002500001070BF36EF80EC715F31055
:1025F000C76F0101010EC86F0001C751070B026EC2
:10260000010EE66ED950020FE66EDACFE6FF010E3C
:10261000B6D0AADB01E1051C04E004EB46F205EBB1
:1026200047F2010EE66E460EE66E020EE66E020EF2
:10263000A6D0016A6851580A4FE00A0A3AE0040A33
:102640002DE01F0A27E01D0A21E0170A1BE00E0AF1
:102650000EE00A0A01E07AD060DB030E025C01E3BF
:1026600040D2E66A0101D9500C0FC9DAF6D755DB22
:10267000030E025C01E335D2E66A0101D950180F5E
:10268000BEDAF6D7B7DA6FEC2EF00BD0B3DA32EC55
:102690002EF007D0AFDA47EC2EF003D0ABDA5FECC8
:1026A0002EF0F3CFE6FFF4CFE6FF13EC38F044E969
:1026B00018D294DB8DEC34F045E902C2E6FF03C288
:1026C000E6FF030E9DDB5DEC36F045E906C2E6FF52
:1026D00007C2E6FF020EA9D08B0EE66E720E8DDBEE
:1026E000ABD0016A680EE66EE66A600EE66E000E1A
:1026F000E66E020EE66E770EE66EA5EC1DF046E97C
:102700000101C85104E0FAEC1CF00101C86BC95189
:10271000CA1101E1E6D1020EC96FCA6BE2D1300ED7
:10272000695D026E0250090802E2070E025E025065
:102730000F0802E2200E025E02500F0801E2D1D122
:10274000016A68514D0A0FE00A0A02E00168C9D126
:1027500024DB900E0101CC27000E69DA900E0101F6
:10276000CC27000E0AD019DB600E0101CC27000E29
:102770005EDA600E0101CC27000E2ADB040E08DBB6
:10278000B0D1D950040F33DA61DD44E9016E015054
:1027900001E0A7D10001C751070B010A3CE0010A83
:1027A0003AE0020A1BE0010A07E0070A01E099D1BA
:1027B0002DDA13EC1FF032D029DA13EC1FF046E9C2
:1027C000810EE66E720E1FDB88DA040E19DB8ADAE0
:1027D000040EE66E8D0EE66E010E2BD009DB79DA63
:1027E00074DA78EC1FF046E9026A060E025C10E229
:1027F000090E0202F350036EE66A0101D9500C0F74
:10280000A2DA0350B8DA76DA200EEF6E022AEDD79C
:1028100071DAEF6A66D1FAD9B0EC1EF046E9DEDA79
:102820005CDA030EEDDA5EDA030EE66E8C0EE66E0F
:10283000010EE66E96EC36F045E953D1520E685D16
:1028400001E04FD1470E695D01E04BD1010EC96F28
:10285000CA6B016A46D1020EF66E770EF76E09005A
:10286000F5CF60F00900F5CF61F00900F5CF62F017
:102870000900F5CF63F00900F5CF64F00900F5CF4A
:1028800065F00900F5CF66F00900F5CF67F00900A3
:10289000F5CF68F00900F5CF69F00900F5CF6AF0CF
:1028A0000900F5CF6BF00900F5CF6CF00900F5CF0A
:1028B0006DF00900F5CF6EF00900F5CF6FF009005B
:1028C000F5CF70F00900F5CF71F00900F5CF72F087
:1028D0000900F5CF73F00900F5CF74F00900F5CFCA
:1028E00075F00900F5CF76F00900F5CF77F0090013
:1028F000F5CF78F00900F5CF79F00900F5CF7AF03F
:102900000900F5CF7BF00900F5CF7CF00900F5CF89
:102910007DF00900F5CF7EF00900F5CF7FF00900CA
:10292000F5CF80F00900F5CF81F00900F5CF82F0F6
:102930000900F5CF83F00900F5CF84F00900F5CF49
:1029400085F00900F5CF86F00900F5CF87F0090082
:10295000F5CF88F00900F5CF89F00900F5CF8AF0AE
:102960000900F5CF8BF00900F5CF8CF00900F5CF09
:102970008DF00900F5CF8EF00900F5CF8FF009003A
:10298000F5CF90F00900F5CF91F00900F5CF92F066
:102990000900F5CF93F00900F5CF94F00900F5CFC9
:1029A00095F00900F5CF96F00900F5CF97F00900F2
:1029B000F5CF98F00900F5CF99F00900F5CF9AF01E
:1029C0000900F5CF9BF00900F5CF9CF00900F5CF89
:1029D0009DF00900F5CF9EF00900F5CF9FF00900AA
:1029E000F5CFA0F00900F5CFA1F00900F5CFA2F0D6
:1029F0000900F5CFA3F00900F5CFA4F00900F5CF49
:102A0000A5F00900F5CFA6F00900F5CFA7F0090061
:102A1000F5CFA8F00900F5CFA9F00900F5CFAAF08D
:102A20000900F5CFABF00900F5CFACF00900F5CF08
:102A3000ADF00900F5CFAEF00900F5CFAFF0090019
:102A4000F5CFB0F00900F5CFB1F00900F5CFB2F045
:102A50000900F5CFB3F00900F5CFB4F00900F5CFC8
:102A6000B5F00900F5CFB6F00900F5CFB7F00900D1
:102A7000F5CFB8F00900F5CFB9F00900F5CFBAF0FD
:102A80000900F5CFBBF00900F5CFBCF00900F5CF88
:102A9000BDF00900F5CFBEF00900F5CFBFF0090089
:102AA000F5CFC0F00900F5CFC1F00900F5CFC2F0B5
:102AB0000900F5CFC3F00900F5CFC4F00900F5CF48
:102AC000C5F00900F5CFC6F00800F5CFC7F0C86B18
:102AD000CB6B010EC91904E1CA5102E1C96BCA6B83
:102AE000016A015064E9E7CFD9FF1200B7D881E944
:102AF00043E88DDC016E015042E00A0EE66E670E7F
:102B0000E66E010EE66E79EC34F043E9F350026EA6
:102B1000F450036E0150010187271F0EE76E8719DD
:102B200002E7E73402D0E750875D09E3010EF36E58
:102B3000F46AF3508708026E010EF454036E0250DB
:102B400003101DE002EBE9FF03EBEAFFEF6A7FDC15
:102B5000000906E0ED0EE66E7D0EE66E000E05D075
:102B6000E80EE66E7D0EE66E000E4AD95DEC34F09E
:102B700045E90101876B77D80201010EB46F0201AC
:102B8000B45101E058DC44E9E7CFD9FF12003CEC36
:102B900037F05EEC37F00201A651030827E2060E7B
:102BA000A65D24E3A3DF02EC32F00101CA3508E29E
:102BB000C9510108000ECA5503E2C92B000ECA23F1
:102BC0000A0EC91913E1CA5111E1E668E66AF9EC87
:102BD0001DF042E95CEC37F00101C96BCA6BC90713
:102BE000000ECA5BC951CA11FAE12FDC1200ECD801
:102BF000D4EF16F0880EE66E010EE66E1200A3D832
:102C0000090E0202F350B7D8022A1200F1D8D950A7
:102C1000060FDAD8D950040FE4EF16F0E66EC4D8E8
:102C2000EFEC10F044E9016E010EE66E1200D0D810
:102C3000BBD850EC11F044E9016E010EE66ECDEF09
:102C400016F002EBE9FF03EBEAFFEF501200A4ECF1
:102C500011F044E9016EFF0E025C1200D9CFE6FFCD
:102C6000E1CFD9FF1200200EE66EE66AE66A670E33
:102C7000E66E010EE66E1FEC34F045E9120000EB43
:102C8000E9FF01EBEAFF1200D950050F9DD802EBD6
:102C9000E6FF03EBE6FF120001010224CC6F000EF9
:102CA0000320CD6FCCC1E6FFE66E120042E9F3CF00
:102CB000CCF1F4CFCDF10101F350F410120026EC69
:102CC00011F044E9016E041C1200D9500C0FE4EF1E
:102CD00016F0D950180FE4EF16F08DEC34F045E9FA
:102CE000F8EF16F05DEC36F045E906EBE6FF07EB92
:102CF000E6FF1200080E0324EA6A880FE96E010E4F
:102D0000EA22120001EBE9FF02EBEAFFEFCFCEF17E
:102D1000120043E9E7CFD9FF1200030EE66E010E61
:102D2000E66ED3DFD6DFFFEC1CF046E9980EE66EC8
:102D3000720E63D845E9026A12000268D950020F88
:102D400056DF27EF16F0CE6FDACFCFF10250040D29
:102D5000CE51F324CC6FDA50F420CD6FCCC1E6FF16
:102D6000E66E040EE66E120004680568D950040F82
:102D70003EDF5FEF16F0D16B880FD06F010ED123CD
:102D8000D0C1E6FFD1C1E6FFBBEC36F046E9120048
:102D900037D8BBEC36F046E912000250040DF3CFF1
:102DA000CCF1F4CFCDF11200C1EC11F0F3CFE6FF7E
:102DB000F4CFE6FF1200400EE66EE66AE66A1ADF1E
:102DC0001FEC34F045E91200E66EDACFE6FF1200A0
:102DD000CD23CCC1E6FFCDC1E6FF1200900EE66E1A
:102DE000720E03EF17F03ADF85E942E821EF16F0A3
:102DF00004EBE6FF05EBE6FF120005D88DEF34F09B
:0E2E0000E66EFAEF15F0E66EE66AFAEF15F0F0
:022E0E000000C2
:102E100000000000000000000000000000000000B2
:102E200000000000000000000000000000000000A2
:102E30000000000000000000000000000000000092
:102E40000000000000000000000000000000000082
:0639C00000000000000001
:0A39C6000201000E886F050E896FE4
:1039D000020EE66EF00EE66E460EE66E020EE66E25
:1039E00052D944E90201461D04E1471D02E1466B3C
:1039F000476B12000201466B476BE6EF1FF0EBDBF3
:103A000041E8076AD890075002E6030E075C45E2DA
:103A100000EBE9FF01EBEAFF6FDB0101D56BD4BFDF
:103A2000D569FFDACFAF02D0D069D1690D0E1F0B77
:103A300003E0010168DBFEE107EBCCF10101CD6B96
:103A4000CCBFCD6941DB0224E96ECD51032006DBFA
:103A500000EBE9FF01EBEAFF060EE926000EEA2281
:103A60004BDBD56BD4BFD569DCDACFAF02D0D069E0
:103A7000D1690E0E1F0B03E0010145DBFEE107EBF0
:103A8000CCF10101CD6BCCBFCD691EDB0424E96E06
:103A9000CD510520E3DA072AB5D742E9E7CFD9FFB0
:103AA0001200D9CFE6FFE1CFD9FF85E942E802EB6A
:103AB000F6FF03EBF7FFF86AA68EA69CA684A688FD
:103AC000F250800B01E0010E066EF29E550EA76EBD
:103AD000AA0EA76EA68200000650E8B0F28EE8A0FB
:103AE000F29EA694056A400E055C2BE20550002468
:103AF000E96E000E0120EA6EEF50F56E0D0005280C
:103B00001F0B1DE1200EF65E000EF75A000EF85A4C
:103B1000A68EA69CA684A698F250800B01E0010E0A
:103B2000066EF29E550EA76EAA0EA76EA682000024
:103B3000A694200EF626000EF722000EF822052A83
:103B4000D2D743E9E7CFD9FF120045DB7FE845E84C
:103B50003F0E0414076EC00E0414086EFF0E051409
:103B6000096E400EE66EE66A08EBE6FF09EBE6FF3B
:103B7000E66AD9500B0F24DBFCEC33F047E9005028
:103B8000011026E0D890075002E6400E075C20E2C4
:103B9000C1DAEF50E66E0101D9500B0FCC6FDACFCE
:103BA000CDF107EBCEF1CF6BCEBFCF69CC51CE2597
:103BB000E96ECD51CF21EA6EE552E750EF6E072A4C
:103BC000042A000E0522022A03220006015AD7D732
:103BD000D9500B0FF5DA08EBE6FF09EBE6FF61DFE2
:103BE00044E900500110B4E17FE946E9E7CFD9FF8D
:103BF0001200D9CFE6FFE1CFD9FF83E941E8A6A2C1
:103C000002D00000FCD700EBA9FF01EBA8FFA69EA5
:103C1000A69CA698A684F250800B01E0010E036ECC
:103C2000F29E550EA76EAA0EA76EA6820350E8B0AC
:103C3000F28EE8A0F29EA69442E9E7CFD9FF1200E7
:103C4000EBD984E900EBA9FFA69EA69CA68001EB18
:103C5000E9FF02EBEAFFA8CFEFFF61D2DDD985E9EA
:103C6000005010E003EBE6FF01EBE9FF02EBEAFF97
:103C7000EFCFE6FFBEDF42E90006012A000E022276
:103C8000032AEED74CD2C8D985E943E882EB05F088
:103C900083EB06F081EB07F0A6B2FED7A1980050A7
:103CA0000EE007EBE6FF05EBE6FF06EBE6FFC8DFFD
:103CB00043E90006052A000E0622072AF0D744E948
:103CC000E7CFD9FF1200A8D989E942E8020146519D
:103CD000DC08050E475502E2466B476BB50EE66EF3
:103CE000E66A06EBE6FF07EBE6FFD8EC2CF0E552C0
:103CF000E5500A6EE750096E5A0E01010224CC6F9E
:103D0000000E0320CD6FCC510926CD510A22020EA0
:103D1000E66ED950090F54DA020EE66EE66AA8D9AB
:103D20005DDAA6D909DA0101CC51CD1114E1400EBA
:103D3000E66EE66A16D9400ECC5F000ECD5B010E32
:103D400088D9FEE115DA200ECC5F000ECD5B010EA6
:103D500080D9FEE137D93AD943E9E7CFD9FF12003C
:103D60003ADA42E8C00E87D9C00EB6D910E1CF5179
:103D7000CD190DE102014651005C4751015807E29F
:103D8000020EE66EE66EE66A400E2BD90BD0CBD95A
:103D9000010ED890F636F736E806FBE109DA0A009C
:103DA000F550086EB50E71D9C7D901015A0ECC5F16
:103DB000000ECD5BAFD9CCC1EEFFCDC1EDFFB50E8E
:103DC000E66EE66A62D90101FE0EE350075CCE6F33
:103DD00041E9E5500858CF6FCEC1E6FFE66E17EC1B
:103DE0002CF0AAD904EBE9FF05EBEAFFCCC1EEFF0A
:103DF000CDC1EDFF43E9E7CFD9FF12000DD974D94A
:103E000002E2466B476B49D9FAD847D9BDD809E1D8
:103E1000C8D91FD9FEE1ACD9100E51D91AD9FEE18B
:103E2000D1D8D4D885D1D7D944E8E00E24D9E00E32
:103E300053D910E1CF51CD190DE102014651005C7B
:103E40004751015807E2040EE66EE66EE66A200E60
:103E5000C8D80BD068D9020ED890F636F736E806E7
:103E6000FBE1EFD80800F5500A6E54D909EBEEFFDC
:103E70000AEBEDFF04EBE9FF05EBEAFF07EBEEFFD2
:103E800008EBEDFF55D1C8D82FD902E2466B476B3E
:103E90000DD9B5D80BD978D809E183D9DAD8FEE1A4
:103EA00067D9100E0CD9D5D8FEE18CD88FD840D167
:103EB000B3D883E90C0E88D946C2CCF147C2CDF104
:103EC0000101CD03F3CFCDF1CC03F3CFCCF1F4500E
:103ED000CD270E0E53D90201462B000E4723FA0EB2
:103EE000465D000E475902E3466B476B6FD817D10A
:103EF00072D94CE818D90C0EF702F3CFF7FFF6028F
:103F0000F3CFF6FFF450F7269CD80900F5500A6E5F
:103F10000900F5500B6E0900F5500C6E0900F550C4
:103F20000D6E0900F5500E6E0900F5500F6E090078
:103F3000F550106E0900F550116E0900F550126E23
:103F4000D950070F3DD904EBE6FF05EBE6FF02EB86
:103F5000E6FF03EBE6FF53DD46E94DE9E7CFD9FF86
:103F60001200480EE66E020EE66E8DDE44E9400E4B
:103F7000E66EE66A480EE66E020EE66E46C2CCF1CA
:103F800047C2CDF10101120000EBE6FF01EBE6FFB5
:103F900002EBE6FF03EBE6FFDDD80B6ECF510C6EB4
:103FA000040EE66ED950090F0BD9040EE66EE66AD0
:103FB000200EC8D813D9200EC5D8BED80101CC51C7
:103FC000CD1112000E0E0101BEEF20F0020EE66EC2
:103FD000460EE66E020EE66EF00EE66E3FDE44E939
:103FE0001200F2D81AEC2CF0D8EC2CF0A5D8CCC1E9
:103FF000E6FFD950070FE4D846DE44E9120004EB8F
:10400000E6FF05EBE6FF06EBE6FF07EBE6FFA2D8CF
:10401000096ECF510A6E1200D9CFE6FFE1CFD9FF6A
:104020001200D890D437D537D251D425E96ED35168
:10403000D521EA6EEECFCEF1EFCFCFF1D06BD16BC1
:104040001200B6D80900F550086E0900F550096E47
:104050001200D890CC37CD37E8061200EA6ECEC1F8
:10406000EEFFCFC1EEFFD0C1EEFFD1C1EEFF1200D7
:10407000400EA2EF20F0020146150101CC6FFF0EA9
:10408000020147150101CD6F1200E66EE66A07EBEB
:10409000E6FF08EBE6FF1AEF2CF0E0C1E6FFE1C116
:1040A000E6FFE2C1E6FFE3C1E6FF1200DCC1E6FF86
:1040B000DDC1E6FFDEC1E6FFDFC1E6FF1200CC5F37
:1040C000000ECD5B020E1200D890CC37CD37D890C1
:1040D000CC37CD37CC5112000014CE6FFF0E011437
:1040E000CF6FCE51CC19120089E944E80201465144
:1040F000EE08020E47551200E9CFD2F1EACFD3F114
:1041000007EBD4F11200D890CE37CF37D037D13764
:10411000E806120002EBE9FF03EBEAFF120041E9B7
:10412000E7CFD9FF120000EBF6FF01EBF7FF12001B
:1041300045E9E7CFD9FF1200E552E5CFCDF1E7CF52
:10414000CCF11200E66EE66A46C2E6FF47C2E6FF21
:104150001AEF2CF00DEC35F048E9A2C2CCF1A3C265
:10416000CDF1A4C2CEF1A5C2CFF10101CE51120012
:1041700029DF400EE66EE66EB1EF1FF0CC272E0E63
:10418000CD23CCC1E6FFCDC1E6FFDFDC46E912005E
:10419000CCC1E6FF63DD44E90201462B000E472354
:1041A0001200400EE66EE66ADCDE200E5FEF20F0C5
:1041B0000E0EF6262E0EF7220900F550076E12009D
:1041C000E66EDACFE6FF1200E66EE66A00EBE6FF87
:1041D00001EBE6FF120020DF87E91200D8EC2CF09B
:0641E000ABDFC8EF20F088
:0A41E600800EC76E280EC66E180E7C
:1041F000C86EC56A800EE66E080EE66ED0EC3DF025
:1042000042E90101636B646B006B016B010E026F8D
:10421000656B666B8A8A8996536B546B556B566BCC
:1042200053C14FF154C150F155C151F156C152F132
:1042300053C14BF154C14CF155C14DF156C14EF132
:10424000120078DA82E941E80050E824900F026E0B
:10425000C7EC15F0E6EC3EF0C580C5B0FED702EB2A
:10426000E6FF76DAC5AC02D0000E07D09F0EE66EF0
:104270006FDAC584C5B4FED7010EF36EF46A42E965
:10428000E7CFD9FF120056DA84E946E80250E82465
:10429000910F046E800E076EC7EC15F0E6EC3EF051
:1042A000C580C5B0FED704EBE6FF52DAC5BC27D007
:1042B000030EE66ED950050FE66EDACFE6FFA3ECEB
:1042C0003CF043E9E6EC3EF0C58AC588C5B8FED7A8
:1042D000C584C5B4FED705EBCEF1CEC1CFF1010147
:1042E000CE6B0650CE25CC6F000ECF21CD6F00EBEC
:1042F000E9FF01EBEAFF31DA800E071402E0000E5D
:1043000001D0010E47E9E7CFD9FF120013DA82E9A5
:104310000C0EE66E7F0E0014FE0BFD0BE66EAD0E6E
:10432000E66E46EC3CF043E9010E1CDA0FEC3FF080
:1043300041E9E7CFD9FF1200FDD981E942E8BFEC9E
:104340003EF0000EF35C016E020EF458026E06ECB5
:104350003FF001EBF3FF02EBF4FF43E9E7CFD9FFB6
:104360001200010EE66E6DDF41E9020EE66E69DFB6
:1043700041E9E66A66DF41E98F0EE66EC7DF41E993
:104380001200D8D981E941E819DA01E13CD11EDAFD
:1043900001E139D12BDA01E136D10101005113E0FD
:1043A0005DC157F15EC158F15FC159F160C15AF169
:1043B00061C15BF162C15CF18A9A030ED3D989862F
:1043C0000101006B1CD1016AD890015002E6030E76
:1043D000015C01E3FAD088D9E9BEEA6889D9570EB1
:1043E000E926010EEA22EECFD2F1EFCFD3F17CD94C
:1043F000E9BEEA687DD95D0EE926010EEA22EE509B
:104400000101D25DD06FEE50D359D16FD06DD11F65
:10441000000ED12383D9060EE926000EEA228FD999
:10442000CEBFCF6969D9E668E668E668E66863C129
:10443000D4F164C1D5F1D66BD76BD5AF02D0D669B4
:10444000D769D4C1E6FFD5C1E6FFD6C1E6FFD7C123
:10445000E6FF4AD9E9BEEA684BD94AD93F0EE926B8
:10446000010EEA2284D983D953EC2CF00CEC2DF008
:10447000E552E5CFD3F1E5CFD2F1E5CFD1F1E7CFEA
:10448000D0F14CD95CD9CEBFCF6936D92DD9E9BE90
:10449000EA682ED92DD94B0EE926010EEA22EE6AE2
:1044A000EE6AEE6AEE6A20D9E9BEEA6821D9150EF5
:1044B000E926010EA2D9E9BEEA681AD9210EE92639
:1044C000010EEA228BD9E9BEEA6812D92D0EE9263F
:1044D000010E6BD9E9BEEA680BD9390EE926010E47
:1044E00058D9E9BEEA68FD0EE926000EEA22EFCFB0
:1044F000CEF1CF6BCEBFCF693FD9E9BEEA6884D990
:104500002CD9F2D8E9BEEA68F3D80F0EE926010EDD
:1045100074D9E9BEEA68ECD81B0EE926010EEA223E
:1045200001015CD9E9BEEA68E3D8270EE926010E4D
:104530003CD9E9BEEA68DCD8330EE926010E29D958
:10454000E9BEEA68FA0EE926000EEA22EFCFCEF1C4
:10455000CF6BCEBFCF6910D9E9BEEA68C9D8030EC8
:10456000E926010EEA22F9D80001C751800B24E0A8
:10457000BBD8E9BEEA6848D9FAD843EC36F042E93C
:10458000F3CFCCF1F4CFCDF1140E0101D890CDBF13
:1045900003D0CC5D000ECD590FE2010E01EBF3FF0D
:1045A000015204E0D890E836F306FCE10101651100
:1045B000656F030E662707D00101665102E06605AC
:1045C00001D0000E666F012AFFD6665101E1656BCE
:1045D0008996030EC7D88A8A0101010E006F030E67
:1045E000E66E010EE66E51EC24F042E90101636BC8
:1045F000646B022B0251040802E2010E026FB1DE6D
:104600000101016B19D00101643516E263516408A0
:10461000000E645511E2100E656FD0D802E1010161
:104620006581D4D802E101016583E0D802E101018E
:10463000658501010A0E666FFEEC3EF0000950E14F
:104640007BDEF3CFCCF1F4CFCDF10101CE6BCF6B9C
:10465000CDAF02D0CE69CF6901010151040DF3CF76
:10466000E9FFF4CFEAFF4B0EE926010EEA22010131
:10467000CC51EE26CD51EE22CE51EE22CF51EE227C
:104680000101012B030E015D1CE3016B4BC13FF1E6
:104690004CC140F14DC141F14EC142F14FC143F116
:1046A00050C144F151C145F152C146F153C147F1E6
:1046B00054C148F155C149F156C14AF1632B000E6E
:1046C00064230151020A08E0030A04E0010A08E138
:1046D0008F0E03D0970E01D0870EE66E17DE41E9EC
:1046E00042E9E7CFD9FF120001EBE9FFEA6A1200C5
:1046F000D890E936EA361200D890CE37CF37CC5171
:10470000CE25E96ECD51CF21EA6ED0C1EEFFD1C1E9
:10471000EDFF1200B8DD43E900091200010102516A
:104720000C0DF3CFE9FFF4CFEAFF030EE926010EEB
:10473000EA221200D9CFE6FFE1CFD9FF1200E9CF7C
:10474000CCF1EACFCDF101EBCEF10101CF6B12003C
:10475000F7EC3CF041E9E6EF3EF0CCC1EEFFCDC115
:10476000EDFF1200E66ECBEC3EF041E91200EECF19
:10477000E6FFEECFE6FF1200CEC1E6FFCFC1E6FFB7
:10478000D8EC2CF0E552E5CFCDF1E7CFCCF174EFCA
:1047900023F0EA22D251EE24D06FD351EE20D16F14
:1047A000D0C1E6FFE66E74EF23F0EA22D451EE2486
:1047B000D26FD551EE20D36F74EF23F05D0EE66E0D
:1047C000010EE66E010EE66E8AEF23F05F0EE66ED6
:1047D000010EE66E020EE66E8AEF23F0D651EE244D
:1047E000D46FD751EE20D56F74EF23F0610EE66ED3
:1047F000010EE66EE66A8AEF23F0EA22EECFD6F1EA
:10480000EFCFD7F174EF23F073DF090EE926010E25
:04481000EA22120086
:0C481400D6DA83E941E8036AD89003502B
:1048200002E6180E035C39E2040EE66E03EBE6FFC7
:10483000B4EC2CF041E9E750000906E00101D06B2F
:10484000D16BD26BD36B06D00101D06BD16BD26B25
:10485000010ED36F00EBE9FF01EBEAFFE9CFCCF1EA
:10486000EACFCDF103EBCEF1CF6BCEBFCF69D890BD
:10487000CE37CF37D890CE37CF37CC51CE25E96E53
:10488000CD51CF21EA6ED0C1EEFFD1C1EEFFD2C132
:10489000EEFFD3C1EEFF032AC1D742E9E7CFD9FF2C
:1048A00012008FDA83E945E8036AD890035002E6E4
:1048B000060E035C0EE203EBE9FFEA6AE9BEEA6872
:1048C000A8DA03EBE9FFEA6AE9BEEA68A5DA032A97
:1048D000ECD7E66A00EBE6FF01EBE6FF22EC0CF01A
:1048E00043E92CC2CCF12DC2CDF12EC2CEF12FC2A4
:1048F000CFF1020130510101CC27020131510101F8
:10490000CD23020132510101CE23020133510101B5
:10491000CF233CDA06DAB9EC35F044E949DA0ADAB1
:1049200000DA58DAE5D9010131DA39DA14C2E6FFE2
:1049300015C2E6FF16C2E6FF17C2E6FF18C2E6FF81
:1049400019C2E6FF1AC2E6FF1BC2E6FF54DAA2C292
:1049500000F2A3C201F2A4C202F2A5C203F2020154
:10496000033504E3680E0227010E032318DAD9D9B0
:104970001CC2E6FF1DC2E6FF1EC2E6FF1FC2E6FF25
:104980003ADAA2C204F2A3C205F2A4C206F2A5C298
:1049900007F246E9E7CFD9FF120013DA81E94CE8C4
:1049A000056A066A076A086A0A6A0B6A060ED890E0
:1049B0000BBE03D00A5C000E0B580EE20AEBE9FFB7
:1049C0000BEBEAFF26DA0AEBE9FF0BEBEAFF24DA4E
:1049D0000A2A000E0B22EAD70A6A0B6A380ED89010
:1049E0000BBE03D00A5C000E0B5801E38CD00AEB1F
:1049F000E6FF0AEBCEF10BEBCFF101010C0ECF037A
:104A0000F3CFCFF1CE03F3CFCEF1F450CF27020195
:104A100088510101F324CC6F020189510101CF219A
:104A2000CD6FCCC1E6FFE66E22EC0CF043E9100E30
:104A3000D8900BBE03D00A5C000E0B5860E2030E48
:104A400001010A14CC6FCD6B030ECC1958E1CD5186
:104A500056E1096AD890095002E6030E095C4FE25C
:104A6000020EE66EE66AE66AE66AB0D9E9BEEA6870
:104A700033D9C8D9EFCFE6FF53EC2CF0E552E5CFA0
:104A8000EDFFE5CFEDFFE5CFEDFFE7CFEFFF9ED9DF
:104A9000E9BEEA6821D9EE50016EEE50026EEE508A
:104AA000036EEF50046E92D9E9BEEA68BDD98ED983
:104AB000E9BEEA6893D901EBD0F102EBD1F103EB47
:104AC000D2F104EBD3F182D9E9BEEA680BD944D91B
:104AD000D950050FE96EDACFEAFFCC51EE26CD5161
:104AE000EE22CE51EE22CF51EE2270D9E9BEEA6815
:104AF00093D96CD9E9BEEA688CD9092AABD70A2ABE
:104B0000000E0B226BD7030E0C6ED8900C5002E6F1
:104B1000060E0C5C47E2EDC1E6FFEEC1E6FFEFC119
:104B2000E6FFF0C1E6FF0CEBE9FFEA6AE9BEEA68DE
:104B300055D90CEBE9FFEA6AE9BEEA6875D901EBE1
:104B4000E6FF02EBE6FF03EBE6FF04EBE6FF42D9EC
:104B50002FD90CEBE9FFEA6AE9BEEA68C3D8010184
:104B6000FBD8F1D8D950010FE96EDACFEAFF020E77
:104B7000E76ED890030EEB32020EEB32010EEB32F1
:104B8000EF32E706F6E1D950050FE96EDACFEAFF1A
:104B90000150EE260250EE220350EE220450EE2287
:104BA0000C2AB3D705EBA2F206EBA3F207EBA4F2B3
:104BB00008EBA5F24DE9E7CFD9FF120030D92ADE84
:104BC00042E99FD8EADEA2C20CF2A3C20DF2A4C24F
:104BD0000EF2A5C20FF20201106B116B200E126FC4
:104BE000136B1200EED882E945E802011051111151
:104BF0001211131165E0005002E1010E456F066AC3
:104C0000D890065002E6180E065C4AE27AD80050A8
:104C10000EE006EBE9FFEA6AE9BEEA68AAD8EE26EA
:104C20001151EE221251EE221351EE220DD006EB5D
:104C3000E9FFEA6AE9BEEA689CD8EE5E1151EE5AD5
:104C40001251EE5A1351EE5AA8DE52D80101CC513E
:104C5000026ECD51036ECE51046ECF51056E02012E
:104C60000C51025C0D5103580E5104580F51055858
:104C700015E2600EE66EE66A600EE66E000EE66E07
:104C8000CED8D1EC33F046E902EB0CF203EB0DF297
:104C900004EB0EF205EB0FF20201456B062AB0D7CA
:104CA00045510DE000500BE0010E1F0B08E0020122
:104CB000D8901333123311331033E806F9E121D8B9
:104CC0000CC2A2F20DC2A3F20EC2A4F20FC2A5F250
:104CD00046E9E7CFD9FF120087D8140EE926020E65
:104CE000EA22120081D82C0EE926020EEA221200D6
:104CF000A2C2CCF1A3C2CDF1A4C2CEF1A5C2CFF124
:104D00001200600EE66EE66A8AD8600EE66E000E4D
:104D1000E66ED1EC33F046E9120074D8EECFE6FF30
:104D2000120004EBE6FF05EBE6FF06EBE6FF07EB00
:104D3000E6FF1200A2C2E6FFA3C2E6FFA4C2E6FF9E
:104D4000A5C2E6FF1200CC51016ECD51026ECE51CC
:104D5000036ECF51046E1200D051EE5CCC6FD15176
:104D6000EE58CD6FD251EE58CE6FD351EE58CF6F73
:104D700012003AD8600EE926000EEA220201105114
:104D80001200EE6AEE6AEE6AEE6A1200CC51046E10
:104D9000CD51056ECE51066ECF51076E1200E9C19E
:104DA000E6FFEAC1E6FFEBC1E6FFECC1E6FF120059
:104DB000A2C2D0F1A3C2D1F1A4C2D2F1A5C2D3F153
:104DC0001200D9CFE6FFE1CFD9FF120009EBE9FFCE
:104DD000EA6A12000DEC35F048E9120025D8FADF36
:104DE00087DF0101A3EF26F0D890E936EA36D890A4
:104DF000E936EA361200EBEC29F048E979DF9ADF70
:104E0000EAEF26F0EECFE6FFEECFE6FFEECFE6FFCD
:104E1000120062DFC1EF26F065DFC1EF26F0A00EC1
:0E4E2000E66E070EE66E120057DF8DEF26F0ED
:024E2E00060E6E
:104E3000E66EB6EC3DF041E9400EE66E17EC3CF054
:104E400041E9D70E9314936EDFEC3EF0BA6A8A867E
:104E5000670EE66EE66A3C0EE66E07EC3BF043E951
:104E6000E60EE66E91EC3EF041E96D0EE66E730ED5
:104E7000F6D94A0EE66E730EF2D93D0EE66E730E4B
:104E8000EED92E0EE66E730EEAD9290EE66E730E7B
:104E90002FEF29F0F3D987E9220EE66E730EE66E46
:104EA000E66A1BDA8DEC34F045E9D9CFE9FFDACFB9
:104EB000EAFF080EE76ED890030EEB32020EEB32DB
:104EC000010EEB32EF32E706F6E1E4D9E3D9BED9C1
:104ED0000DEC35F048E9A2C2D0F1A3C2D1F1A4C2D1
:104EE000D2F1A5C2D3F1A2C2E6FFA3C2E6FFA4C2DB
:104EF000E6FFA5C2E6FF0DEC35F048E9A2C2CCF111
:104F0000A3C2CDF1A4C2CEF1A5C2CFF1A4C2E6FFE7
:104F1000A5C2E6FF050EE66EE0D996EC36F045E94F
:104F2000080E7FD9EF6A070E7CD92C0EEF6E050EA6
:104F300078D9EF50E66E060EC9D9EF50E66E050E31
:104F4000C5D92E0EEF6E41E9E7CFD9FF120096D9F1
:104F50008BE956E80B6A97D90D0FADD977D9D9509F
:104F6000170FA9D9180EE66E730EA9D98DEC34F07F
:104F700045E9D9500D0F79D9D950170F76D9120EAE
:104F8000E66E730E9CD95DEC34F045E9010E0C6EB3
:104F90000CEBCCF10101CD6BCCBFCD6984D92A08D3
:104FA0000AE00CEBCCF1CD6BCCBFCD697CD90B18F2
:104FB0000B6E0C2AEDD7E66AD9500B0F93D9010E70
:104FC000E66E0CEBCEF1CF6BCEBFCF690850CE258D
:104FD000CC6F0950CF21CD6FCC2B000ECD23CCC18F
:104FE000E6FFCDC1E6FFBBEC36F046E957E9E7CF77
:104FF000D9FF120043D989E972E828D944D9090FA9
:1050000071D9A5DF4AE9D950090F6CD91DEC3DF0E3
:1050100042E973E9E7CFD9FF120030D982E90050A5
:1050200003E00C0EBA6E02D0BA6A8A860028E86CD9
:10503000E66EE66AD1EC3CF042E941E9E7CFD9FF00
:1050400012001CD983E946E85A0E036E710E046EF5
:10505000050EE66EE66A200E015C0101CC6FCD6B99
:10506000800B01E0CD69CCC1E6FFCDC1E6FFD8ECF5
:105070002CF0E552E550076EE750066E056A050E06
:10508000055C2EE2005022E0040ED8800554CFD8F3
:10509000086E700E0814E8380F0BCD6F070E081459
:1050A000100D080E0814F310CD11086E440E0814EC
:1050B000E840E8403F0BCD6F110E0814040DF3CF0C
:1050C000CCF12A0E0814F310CD1102D00550AFD840
:1050D000086E08EBE6FFE8EC3BF041E9052ACFD784
:1050E00047E9E7CFD9FF1200D9CFE6FFE1CFD9FFDB
:1050F00083E942E8C7EC15F00201D8800B5104E7C0
:10510000C00E0A5DFF0E0B5901E2046A02010B3565
:1051100004E20A514008000E0B5502E2010E046E33
:105120000001C7AB04D0010ED8800454046E000106
:10513000CA5102E1899855D0040EE66EE66A00EB8A
:10514000E6FF01EBE6FFF50EE66E010EE66EB4EC4F
:1051500034F046E9000945E0050EE66EE66A00EB2C
:10516000E6FF01EBE6FFF50EE66E010EE66EDFEC04
:1051700034F046E98998000089880000CAC0E6FF3B
:1051800034D841E900008B9200008B8000000DECC8
:105190003FF00000036A040E035C1EE204500FE0BF
:1051A000010EE66E030ED88003540024E96E000E53
:1051B0000120EA6EEFCFE6FF44DF42E90BD0E66A5A
:1051C00003500024E96E000E0120EA6EEFCFE6FFE7
:1051D00038DF42E9032ADFD7000009EC3FF0000086
:1051E0008B9043E9E7CFD9FF1200D9CFE6FFE1CF9B
:1051F000D9FF82E98B8200008B8000000DEC3FF02C
:105200000000400E00107F0BE66EE8EC3BF041E939
:10521000000009EC3FF000008B9041E9E7CFD9FF97
:1052200012000424E96E000E0520EA6E120001014E
:105230000624CC6F000E0720CD6FCC510324F66EF0
:10524000CD510420F76E0800F550120000EBE6FF88
:1052500001EBE6FF02EBE6FF03EBE6FF1200E66E72
:10526000E66A75EC3CF043E912003CD808EBE6FF37
:1052700009EBE6FF39EC34F044E91200D9CFE6FF40
:10528000E1CFD9FF120029D806EBE6FF07EBE6FFD6
:10529000D9501200E0C1E6FFE1C1E6FFE2C1E6FF3E
:1052A000E3C1E6FF1200CC510824E96ECD5109207C
:1052B000EA6EEF50120016D8EDDD46E91200E66EF8
:1052C000E66A08EBE6FF09EBE6FF1200AADFE5520B
:1052D000E750EF6E040E11EF29F004EBE6FF05EB4B
:0C52E000E6FF1200E66EDACFE6FF1200D7
:0452EC0005DA89E96D
:1052F00045E807340CE3C8D993D97BD9046ECD5166
:10530000056ECE51066ECF51076E010E0D6E033441
:105310000CE327DA006ECD51016ECE51026ECF51F3
:10532000036E010ED8800D540D6E02EBD0F103EB2D
:10533000D1F10101D26BD36BD1AF02D0D269D36965
:10534000D0C1E6FFD1C1E6FFD2C1E6FFD3C1E6FF7F
:1053500067D953EC2CF0E9D9080E1F0B08E00101C6
:10536000D890CC37CD37CE37CF37E806F9E10101F9
:10537000CC5171D90D5001E0E2D909EBA2F20AEB50
:10538000A3F20BEBA4F20CEBA5F246E9E7CFD9FFB1
:105390001200B2D985E944E8033409E200EBA2F235
:1053A00001EBA3F202EBA4F203EBA5F210D0D9D9E2
:1053B000056ECD51066ECE51076ECF51086E05EBCE
:1053C000A2F206EBA3F207EBA4F208EBA5F245E983
:1053D000E7CFD9FF120090D989E959E8216A20D98D
:1053E000D8DF44E9B1D9A2C2E6FFA3C2E6FFA4C256
:1053F000E6FFA5C2E6FF1DD9CCDF44E9E552E7CFC1
:10540000CFF1E552E7CFCEF1E552E7CFCDF1E5524E
:10541000E7CFCCF1A2C2D0F1A3C2D1F1A4C2D2F1A4
:10542000A5C2D3F10101D335CF51D31908E6D0512C
:10543000CC5DD151CD59D251CE59D351CF5904E37E
:10544000EFD8F7D892D905D0F4D8EAD88ED9010E82
:10545000216E0C3401E373D9D2D8D1D890D90D6E16
:10546000CD510E6ECE510F6ECF51106E1CD9950ED0
:10547000CC27DB0ECD23020ECE23F90ECF23CC5149
:10548000FBD8690E156E1F0E166EF30E176E186898
:1054900013D948D9BDD807D9050ECC27000ECD2386
:1054A000CE23CF23CC51E8D807D957D9F30E156EA8
:1054B0008E0E166ED30E5DD908D9CA0ECC272E0ECD
:1054C000CD23D80ECE23020ECF230DEBD0F10EEB61
:1054D000D1F10FEBD2F110EBD3F1DBD805D9B2D873
:1054E0003CD99B0E156EA80E166E250E42D9540E91
:1054F000156EFB0E166EA40E176E186A0DEBE6FF06
:105500000EEBE6FF0FEBE6FF10EBE6FF0BD9ECD856
:10551000DCD8CF2B15EBD0F116EBD1F117EBD2F194
:1055200018EBD3F1B6D8196ECD511A6ECE511B6E51
:10553000CF511C6E19EBE6FF1AEBE6FF1BEBE6FF03
:105540001CEBE6FF90D8D2DE4FD862D8215012E192
:10555000203408E2B50ED06F1F0ED16F920ED26FBD
:10556000010E07D04B0ED06FE00ED16F6D0ED26FD3
:10557000FE0EC7D807340DE204500008000E055493
:10558000000E0654000E075404E27ED86CD831D8C1
:105590003FD8033408E3960ED06FC00ED16FDB0EF8
:1055A000D26FFC0EAED8D880205008E7960E1D5C56
:1055B000C00E1E58DB0E1F58FC0E205809E28ED874
:1055C000D40EEE267E0EEE22480EEE22060EEE22BF
:1055D0001DEBA2F21EEBA3F21FEBA4F220EBA5F24F
:1055E0005AE9E7CFD9FF120048E9AED80101CC5102
:1055F00012000CEC2DF099D80101CC51120009EBEE
:10560000E6FF0AEBE6FF0BEBE6FF0CEBE6FF120012
:105610001D6ECD511E6ECE511F6ECF51206E1200E9
:1056200004EBE6FF05EBE6FF06EBE6FF07EBE6FF24
:10563000120000EBE6FF01EBE6FF02EBE6FF03EBF7
:10564000E6FF120015EBE6FF16EBE6FF17EBE6FFB1
:1056500018EBE6FF1200096ECD510A6ECE510B6EAB
:10566000CF510C6E12001DEBE6FF1EEBE6FF1FEBA9
:10567000E6FF20EBE6FF1200116ECD51126ECE5107
:10568000136ECF51146E1200E668E668E668E668AD
:105690001200D051CC27D151CD23D251CE23D3519A
:1056A000CF23CC51120009EBCCF10AEBCDF10BEB7F
:1056B000CEF10CEBCFF1120011EBE6FF12EBE6FF9F
:1056C00013EBE6FF14EBE6FF120011EBCCF112EB4B
:1056D000CDF113EBCEF114EBCFF11200D9501D0F29
:1056E000E96EDACFEAFF1200156ECD51166ECE517B
:1056F000176ECF51186E1200D9CFE6FFE1CFD9FF58
:105700001200D36FEBDFEE50D05DCC6FEE50D1596D
:10571000CD6FEE50D259CE6FEE50D359CF6FCC51E2
:1057200008EF2BF08FDFBFEF2BF0E552E5CFCFF185
:10573000E5CFCEF1E5CFCDF1E7CFCCF11200A4DF7C
:105740005EDF57DF2BEF2BF0A2C2CCF1A3C2CDF16D
:10575000A4C2CEF1A5C2CFF1120085DF10D808EFA8
:105760002BF092DF66DFF9EF2AF0C0DD3DDF2BEF93
:105770002BF0176E186A43DFD5DF3CEF2BF00DECF2
:0657800035F0F4EF2AF001
:0A57860043E8D9CFE6FFDACFE6FFD3
:10579000E1CFD9FFE2CFDAFF89E9066A1200F3DF31
:1057A000068001D0F0DF01AEDCEF2BF0006C011EB3
:1057B000E86A012206B0067E03AEE4EF2BF0026C2D
:1057C000031EE86A0322067E1CEC2CF003BE06EFE3
:1057D0002CF006AE08D0026C031EE86A0322046CAB
:1057E000051EE86A052206B006D084EB00F085EBC2
:1057F00001F006A004D082EB00F083EB01F0E5524B
:10580000E5CFDAFFE7CFD9FF45E9000C06BEEBEFA5
:105810002BF0E9DFFF0C43E8D9CFE6FFDACFE6FF54
:10582000E1CFD9FFE2CFDAFF89E9066A1200F3DFA0
:10583000068003D0F0DF01D00682056A046A100EEC
:10584000E76ED89002360336043605360050045C05
:105850000150055805E30050045E0150055A022A24
:10586000E72EF0D706B2120006B006D084EB00F0A7
:1058700085EB01F006A004D082EB00F083EB01F091
:10588000E552E5CFDAFFE7CFD9FF45E9120045E859
:10589000D9CFE6FFDACFE6FFE1CFD9FFE2CFDAFFDB
:1058A0008FE90C6A1200F3DF0C8001D0F0DFE86AA8
:1058B00003AE64EF2CF0006C011E021E031E0122D9
:1058C000022203220CB00C7E07AE6FEF2CF0046CAA
:1058D000051E061E071E0522062207220C7E9CECD2
:1058E0002DF007BEA0EF2CF00CAE0FD0046C051EFF
:1058F000061E071EE86A052206220722086C091EFA
:105900000A1E0B1E09220A220B220CB00AD088EBB9
:1059100000F089EB01F08AEB02F08BEB03F00CA0B6
:1059200008D084EB00F085EB01F086EB02F087EB0A
:1059300003F0E552E5CFDAFFE7CFD9FF49E9000CE4
:105940000CBE76EF2CF0E1DFFF0C42E8D9CFE6FF8A
:10595000DACFE6FFE1CFD9FFE2CFDAFF86E9036ACB
:105960001200F3DF038001D0F0DF00AE03D0006C43
:1059700003B0037E01AE02D0016C037E6EEC2DF00D
:1059800001BED4EF2CF003AE02D0016C026C03B068
:1059900081EB00F003A082EB00F0E552E5CFDAFFE7
:1059A000E7CFD9FF43E9000C03BEEFD7F0DFFF0CD0
:1059B00044E8D9CFE6FFDACFE6FFE1CFD9FFE2CF67
:1059C000DAFF8AE980EB04F081EB05F082EB06F068
:1059D00002500402F450016EF350006E0350076E43
:1059E0000502F450036EF350026E07500402F350A8
:1059F0000126F4500222E86A032206500502F35001
:105A00000126F4500222E86A0322E552E5CFDAFFCC
:105A1000E7CFD9FF46E9000C44E8D9CFE6FFDACF5B
:105A2000E6FFE1CFD9FFE2CFDAFF8EE980EB08F0A5
:105A300081EB09F082EB0AF083EB0BF004500802D3
:105A4000F350006EF450016E04500902F350012629
:105A5000000EF420026E04500A02F3500226000EDB
:105A6000F420036E04500B02F35003260550080285
:105A7000F3500126F4500222000E032205500902C1
:105A8000F3500226F450032205500A02F350032675
:105A900006500802F3500226F45003220650090271
:105AA000F350032607500802F3500326E552E5CFD2
:105AB000DAFFE7CFD9FF48E9000C42E8D9CFE6FF8B
:105AC000DACFE6FFE1CFD9FFE2CFDAFF86E9036A5A
:105AD0001200F3DF038003D0F0DF01D00382026AFB
:105AE000080EE76ED890013602360050025C02E3E1
:105AF000026E012AE72EF7D703B2120003B081EB42
:105B000000F003A082EB00F0E552E5CFDAFFE7CF2B
:105B1000D9FF43E9120045E8D9CFE6FFDACFE6FF27
:105B2000E1CFD9FFE2CFDAFF8FE90C6A1200F3DF91
:105B30000C8003D0F0DF01D00C820B6A0A6A096A7C
:105B4000086A200EE76ED89004360536063607360A
:105B5000083609360A360B360050085C01500958E1
:105B600002500A5803500B5809E30050085E0150D8
:105B7000095A02500A5A03500B5A042AE72EE4D756
:105B80000CB212000CB00AD088EB00F089EB01F0E7
:105B90008AEB02F08BEB03F00CA008D084EB00F052
:105BA00085EB01F086EB02F087EB03F0E552E5CFE1
:0A5BB000DAFFE7CFD9FF49E9120040
:065BBA00020EE66EF20E81
:105BC000E66E9D0EE66E020EE66E43EC1EF044E9B4
:105BD0009DC29FF29EC2A0F21200200EE66E310E10
:105BE00067D9440EE66EFE0E63D9020EE66EA2EC95
:105BF0003EF041E9B40EE66EFE0E5AD987D9020195
:105C00009D6BF60E9E6F64EF2FF059D982E944E840
:105C1000046A056A020EE66ED950020FE66EDACF0C
:105C2000E6FF00EBE6FF680EE66E6FEC3AF045E942
:105C3000000913E1FF0E01010214CD6BCD6FCC6B97
:105C4000000E0214FF0E0314CF6FCE6FCF6BCE5138
:105C5000CC11046ECD51CF11056E04EBF3FF05EBB3
:105C6000F4FF5AD1E66A010EE66E180E70D9F3CF32
:105C7000E6FFF4CFE6FFCFEC2BF0E552E5CFCDF118
:105C8000E7CFCCF1CCC1F3FFCDC1F4FF120017D99F
:105C900081E948E845D9056AC00E066E076A086AB8
:105CA0000E0E28D905EBE6FF06EBE6FF07EBE6FF55
:105CB00008EBE6FFEAD849E9E7CFD9FF1200FFD8A1
:105CC00081E944E82DD90C0E15D9AAC2E6FFABC272
:105CD000E6FFACC2E6FFADC2E6FFD7D81DD1100E7D
:105CE000A7EF2FF0ECD883E9010101EBCCF1CD6BEC
:105CF000CCC1E6FF100EDCD800EBE6FF110ED8D8C1
:105D000041E9E7CFD9FF1200800EE66E080ED0D829
:105D1000E7D801E0000C010CD2D881E944E8DFDFCC
:105D2000EFD8CE6BCF6BCDAF02D0CE69CF69FDD8A7
:105D30009DC2CCF19EC2CDF1CE6BCF6BCDAF02D068
:105D4000CE69CF69CF350450CF1908E6CC51015C3C
:105D5000CD510258CE510358CF51045804E201EB03
:105D60009DF202EB9EF2ABDFCBD8D890F45004E664
:105D7000800ECC5D0C0ECD5907E201EB9DF202EBDB
:105D80009EF20201A1693BD0043401E2C9D8640E3D
:105D9000D06FD16BD26BD36B9DC2D8F19EC2D9F1BB
:105DA000DA6BDB6BD9AF02D0DA69DB69D8C1E6FF09
:105DB000D9C1E6FFDAC1E6FFDBC1E6FFE66EE66ABF
:105DC000E66AE66ABBD80CEC2DF053EC2CF0E552F9
:105DD000E5CFD7F1E5CFD6F1E5CFD5F1E7CFD4F1D7
:105DE0000101D451D05DCC6FD551D159CD6FD65171
:105DF000D259CE6FD751D359CF6FCCC1A1F28CD02D
:105E00005ED882E941E8E66A0DEC28F041E9E66AED
:105E1000F5EC28F041E9005008E0E66A80EC3DF03E
:105E200041E9E66A80EC3DF041E95AD821E00201FF
:105E30009F519D1902E1A0519E1901E045D84FDF05
:105E40005FD8F43406E2CC510008000ECD5501E2D3
:105E50005DD8E668AA0EE66EF9EC1DF042E90BEC9F
:105E60003FF093909392080E8A6E816ED190FFD787
:105E7000E6680DEC28F041E93F0EE66EF5EC28F0FF
:105E800041E942E9E7CFD9FF120058D80DEC35F0CF
:105E900048E9A2C2CCF1A3C2CDF1A4C2CEF1A5C201
:105EA000CFF1010142D803EBF3FF04EBF4FF120042
:105EB000E66E680EE66E48EC3BF043E91200D9CF7F
:105EC000E6FFE1CFD9FF1200020EE66E9D0EE66EF0
:105ED000020EE66EF20EE66E2EEC1EF044E91200A3
:105EE000080EE66E680EE66EBCEC3AF042E9F3503E
:105EF000800B12002CD8F350036EF450046E120085
:105F0000F3CFCCF1F4CFCDF101011200000EE66E1B
:105F1000E66AE8DE42E9120045E9E7CFD9FF120060
:105F2000016A026A036A046A1200CC51016ECD5103
:105F3000026ECE51036ECF51046E120001EBE6FFEC
:105F400002EBE6FF03EBE6FF04EBE6FF1200E66E72
:065F50005CDE41E91200D5
:0A5F56006C5007E1689667D902E17C
:105F60000AD8010C37D8010C040E6C5C03E168966A
:105F700040D8010C000C54D941E8040104BF046B63
:105F800002019C6B946B956B9A6B9B6B90EC32F05F
:105F9000016A010E52D919E20201955116E1F76A20
:105FA0000134FE0BF66EF7363E0EF626740EF7221F
:105FB0000900F5CFCCF10800F5CFCDF1CDC1FAFF46
:105FC0000101CC511400012AE4D7A3D842E9E7CF5C
:105FD000D9FF1200020E0201945D09E170D804019C
:105FE00000BD02D0C80E01D0880E006F1200C2EFB3
:105FF00030F0040E0201A65D09E122C46EFF6E506E
:10600000000802E2050E01D0030EA66F02019405FE
:1060100010E111D8020E02019C5D03E10401840E1F
:1060200006D0040104BD02D0C80E01D0880E046F52
:106030001200C2EF30F0F4D842E80201200E9A5D5F
:10604000000E9B590DE29A51016E9B51026E9C51BC
:1060500002E1010E03D09C0506E1020E9C6F03D005
:10606000200E016E026A040104930491025004138D
:1060700001EB05F4015002019A5F02509B5B400E58
:10608000986F040E996F0201A7A30BD00150021064
:1060900012E096C2F6FF97C2F7FF0800F550B0D89D
:1060A000F5D70150021007E096C2E9FF97C2EAFF58
:1060B000EF50A6D8F6D743E9E7CFD9FF1200B0D802
:1060C00042E8030E04010015026E0151016E9A0EA2
:1060D000E96E020EEA6E0201EE5001249A6FED5055
:1060E00002209B6F400E966F040E976F01500210B6
:1060F0000CE096C2E9FF97C2EAFFEF5098C2E9FFB1
:1061000099C2EAFFEF6EA0D8F1D743E9E7CFD9FFF4
:1061100012006D980201955105E17AD8840E006F46
:1061200004011DD0040120AF1CD002019A510401CA
:10613000265D02019B510401275904E226C49AF20C
:1061400027C49BF278DF0201010E946F61D8800EA4
:10615000006F0401400E066F040E076FC80E046F37
:1061600012000201020E946F0401056BC80E046F49
:106170000401200E016F400E026F040E036FC80E63
:10618000006F12004DD841E8020E0201945D2DE12E
:106190006D50100B2AE0040101510101CC6FCD6B51
:1061A000200ECC1922E1CD5120E140D81EE1005152
:1061B000800B1BE1200E026F040E036F016A200E9C
:1061C0003CD81AE20150EA6A400FE96E040EEA2256
:1061D000EF50E66E0150EA6A200FE96E040EEA22E3
:1061E000E552E750EF6E012AEAD70201946B10D80E
:1061F0008C0E006F0401046B42E9E7CFD9FF120057
:1062000098C2E9FF99C2EAFFEF6E020124EF31F074
:106210000401200E016F200E026F040E036F1200A6
:10622000D9CFE6FFE1CFD9FF81E912000401005187
:106230003C0BE842E8420D081200F36EF46AF3509A
:10624000015C000EF4541200982B000E9923962B3B
:0862500097230106025A120017
:08625800040120511F0B010895
:1062600001E012002051600BE842E842E842E842B7
:10627000E842010801E01200245103E0240501E096
:1062800012002151230A39E0010A33E0030A25E014
:10629000010A1CE0240A31E0070A2FE0010A2DE080
:1062A000030A0EE0010A01E0120031D90201F20EE8
:1062B000966F000E976F0201A7930201080E17D088
:1062C00026D90201F20E986F000E05D020D90201E6
:1062D000EA0E986F000E996F120019D90201EA0EAA
:1062E000966F000E976F0201A7930201070E9A6F37
:1062F00012000DD922C4F1F0120012000001EA6B65
:10630000C20EEB6F010EEC6FED6BEE6BEF6B080ED8
:10631000F06FE36BE26B1A0E726E1E0E736E040169
:10632000600E166F040E176F400E146F0401196F84
:10633000680E1A6F040E1B6F880E186F0401A80EEA
:106340001E6F040E1F6F400E1C6F1200E4D884E90C
:106350000001E26B040118BF24D00050195D02E275
:106360001951006E0001E26B0050E25D13E2E25150
:10637000EA6A680FE96E040EEA22EF50E66EE25117
:106380000124E96E000E0220EA6EE552E750EF6E3E
:10639000E22BEAD70401400E196F1817187D880EFA
:1063A00018130001E25141E9E7CFD9FF12009ED84E
:1063B00012E1036AA1D802E1F45009E000EBE9FF21
:1063C00001EBEAFF002A000E0122EF50F3E176D83C
:1063D000E96B010EE36F97D089D813E1036A8CD87B
:1063E00002E1F4500AE000EBF6FF01EBF7FF002AB0
:1063F000000E01220800F550F2E160D8010EE96FAD
:10640000E36F81D088D881E941E804011CBF55D0F1
:10641000030E0001E35D01E1E36BE3514EE0020E88
:10642000E35D03E104011D6B3FD0E30540E1E8516A
:106430000101CC6FCD6BCC514008000ECD5502E26E
:10644000400E02D00001E851016E01EB1DF4015035
:106450000001E85DE86FA80EE66F040EE76FE9053E
:106460000AE1015011E0E4C0F6FFE5C0F7FF0800C3
:10647000F55030D8F6D7015007E0E4C0E9FFE5C099
:10648000EAFFEF5027D8F7D70001E85110E10401E7
:106490001D510101CC6FCD6B400ECC1905E1CD51E2
:1064A00003E10001020E02D00001030EE36F400E73
:1064B00004011C171C7D880E1C1325D00350005EA0
:1064C000000E015A00EBE4F001EBE5F003EBE8F01D
:1064D00000011200E6C0E9FFE7C0EAFFEF6EE62B1D
:1064E000000EE723E42BE5230106120014D883E90C
:1064F00041E80001E3511200032AFF0EF36EF46A33
:10650000F3500318120042E9E7CFD9FF120002014D
:10651000030E956F1200D9CFE6FFE1CFD9FF12002D
:1065200004012051600BE842E842E842E842E842B8
:10653000000901E012002151070A3FE00B0A3DE08B
:10654000070A32E0010A23E00B0A1FE0020A1DE0FD
:10655000030A19E0080A10E0010A0CE00F0A08E03B
:10656000030A01E0120015D90201040EA66F120001
:10657000DEEF32F015EF33F00CD90201A80E966F62
:10658000020E976F0BD036EF33F068EF33F005D97A
:106590000201976BA90F966F020E97230201A79332
:1065A0000201010E9A6F1200F8D8EA6AA90FE96E8B
:1065B000020EEA2222C4EFFF12001200800E040134
:1065C000205D32E12351030A1FE0010A0AE0030AB9
:1065D00029E1DFD80201730E966F730E976F120ECA
:1065E0001ED0C6D8340EF626740ECBD8020E020189
:1065F000F76A9625F66E9751F7220900F5CF9AF2C1
:106600000A00F5CF9BF20ED0B3D8380EF626740EE2
:10661000B8D896C2F6FF97C2F7FF0800F5500201FE
:106620009A6F9B6B0201A7831200B3D80F0EE66E20
:10663000710EE66E0F0EE66E01EC38F043E9010EC6
:10664000E66EA90EE66E020EE66E01EC38F043E946
:1066500022C4A8F20401225104E10201050EA66F32
:1066600012000201060EA66F7EEF31F00401406BAE
:10667000416B040120511F0B020A0FE0030A0BE0DB
:10668000010A18E186D8040140810201A7A112D0B5
:10669000040140830FD07DD80DD050D801E0010E09
:1066A0005BD898C2E9FFEA6EEF50040B03E00401E7
:1066B000010E406F020195050AE10201400E966F3E
:1066C000040E976F0201A7930201020E9A6F120047
:1066D000040122050EE120511F0B00090AE159D8DF
:1066E000030E0401215D03E10201A78102D0020132
:1066F000A7910401225121E120511F0B02081DE145
:1067000024510F0B000919E019D801E0010E24D81B
:10671000030E0401215D02E1840E03D024AF07D0F3
:10672000400E98C2E9FF99C2EAFFEF6E1200880E90
:1067300098C2E9FF99C2EAFFEF6E12002ED80F0B44
:10674000080DF3500101CD6B000FCC6F040ECD236B
:1067500004012451800B1200040DF3500101CC25DB
:106760000201986F000E0101CD210201996F120004
:1067700010D804012251F66EF76AD890F636F73633
:106780001200F7220900F5CF96F20A00F5CF97F232
:1067900012000201010E956F1200FBDF040124516B
:0267A0001200E5
:0E67A200D9CFE6FFDACFE6FFFA0EE3CFD9FF3C
:1067B000FB0EE3CFDAFFFC0EE3CFE9FFFD0EE3CFE4
:1067C000EAFFE9CFF3FFEACFF4FFF80EE35003E16D
:1067D000F90EE35008E0F80EE30602E2F90EE306D4
:1067E000DECFEEFFF2D7FF0EE3CFDAFFE552FF0E6A
:1067F000E3CFD9FFE5521200FB0EE3CFF6FFFC0E0C
:10680000E3CFF7FFFD0EE3CFF8FFFE0EE3CFE9FF86
:10681000FF0EE3CFEAFFE9CFF3FFEACFF4FFF90E73
:10682000E35003E1FA0EE35009E0F90EE30602E259
:10683000FA0EE3060900F5CFEEFFF1D71200FE0EC7
:10684000E3CFE9FFFF0EE3CFEAFFE9CFF3FFEACFA3
:10685000F4FFFB0EE35003E1FC0EE35009E0FB0EF6
:10686000E30602E2FC0EE306FD0EE350EE6EF1D706
:106870001200D9CFE6FFDACFE6FFFA0EE3CFD9FF59
:10688000FB0EE3CFDAFFFC0EE3CFE9FFFD0EE3CF13
:10689000EAFFE9CFF3FFEACFF4FFEE66FED7ED5251
:1068A000DFCFEEFFDE66FCD7FF0EE3CFDAFFE55267
:1068B000FF0EE3CFD9FFE5521200FB0EE3CFF6FF48
:1068C000FC0EE3CFF7FFFD0EE3CFF8FFFE0EE3CFA4
:1068D000E9FFFF0EE3CFEAFFE9CFF3FFEACFF4FFD2
:1068E000EE66FED7ED520900F5CFEFFFEE66FBD75F
:1068F0001200FE0EE3CFE9FFFF0EE3CFEAFFFD0E2D
:10690000E350EF5C05E0EE66FAD7F36AF46A04D070
:10691000E9CFF3FFEACFF4FF1200FB0EE3CFF6FF5F
:10692000FC0EE3CFF7FFFD0EE3CFF8FFFE0EE3CF43
:10693000E9FFFF0EE3CFEAFFE9CFF3FFEACFF4FF71
:106940000900F5CFEFFFEE66FBD71200FE0EE3CF96
:10695000E9FFFF0EE3CFEAFFF36AF46AEE5203E0C9
:10696000F34AF42AFBD71200D9CFE6FFDACFE6FFCD
:10697000FA0EE3CFD9FFFB0EE3CFDAFFFC0EE3CF35
:10698000E9FFFD0EE3CFEAFFF80EE35003E1F90E55
:10699000E3500AE0F80EE30602E2F90EE306DE50E9
:1069A000EF5C02E1EE66F0D7F36EFF0EE3CFDAFFA5
:1069B000E552FF0EE3CFD9FFE552F3501200D9CFD5
:1069C000E6FFDACFE6FFFA0EE3CFD9FFFB0EE3CF07
:1069D000DAFFFC0EE3CFE9FFFD0EE3CFEAFFE9CFDC
:1069E000F3FFEACFF4FFF80EE35003E1F90EE350B2
:1069F0000BE0F80EE30602E2F90EE306DECFEFFF4E
:106A0000EE66F1D7DD52EFD7FF0EE3CFDAFFE552A6
:0A6A1000FF0EE3CFD9FFE55212009C
:066A1A000BD8E552E5CFA8
:106A2000A5F2E5CFA4F2E5CFA3F2E7CFA2F248E8C2
:106A3000000C46E8D9CFE6FFDACFE6FFE1CFD9FF79
:106A4000E2CFDAFF90E90A6A0B6A0C6A0D6A00501D
:106A50000502F450086E01500402F4500826000E9E
:106A6000096A092200500602F3500826F450092250
:106A7000000E0A2201500502F3500826F4500922A4
:106A8000000E0A2202500402F3500826F450092294
:106A9000000E0A2200500702F3500926F4500A2281
:106AA000000E0B2201500602F3500926F4500A2270
:106AB000000E0B2202500502F3500926F4500A2260
:106AC000000E0B2203500402F3500926F4500A2250
:106AD000000E0B2201500702F3500A26F4500B223D
:106AE000000E0C2202500602F3500A26F4500B222C
:106AF000000E0C2203500502F3500A26F4500B221C
:106B0000000E0C2202500702F3500B26F4500C2208
:106B1000000E0D2203500602F3500B26F4500C22F7
:106B2000000E0D2203500702F3500C26F4500D22E4
:106B3000000E0E2207AE06D000500A5E01500B5A1E
:106B400002500C5A03AE06D004500A5E05500B5A90
:106B500006500C5A89EB00F08AEB01F08BEB02F047
:106B60008CEB03F0E552E5CFDAFFE7CFD9FF4AE936
:106B7000000C0AD844E9E6CFA2F2E6CFA3F2E6CFB2
:106B8000A4F2E6CFA5F2000C46E8D9CFE6FFDACFB3
:106B9000E6FFE1CFD9FFE2CFDAFF8CE944E80366F4
:106BA00024D082EB09F0010E0F6E200E0E6E0D6ADE
:106BB0000C6A010E076E800E066E056A046A040EEA
:106BC000086E09361FE2093609E384EB0CF085EB09
:106BD0000DF086EB0EF087EB0FF014D0D8900E3648
:106BE0000F3606360736082EECD7660E83EB09F013
:106BF000094ECD0E094EA60E094E880E0E6E0C6A79
:106C00000D6A0F6A080E0201B567B551086E0CEBEC
:106C1000E6FF0DEBE6FF0EEBE6FF0FEBE6FF00EB0A
:106C2000E6FF01EBE6FF02EBE6FF03EBE6FF0CEB12
:106C3000E6FF0DEBE6FF0EEBE6FF0FEBE6FF19ECD0
:106C400035F019EC35F0000ED8801056115612565A
:106C5000030E135619EC35F0D8900F320E320D3268
:106C60000C32082ED4D7E552E550036EE550026E83
:106C7000E550016EE750006EE552E5CFDAFFE7CF51
:066C8000D9FF46E9000CFB
:0A6C8600ECD883E901340AE300EBC7
:106C9000CCF101EBCDF10101CC6DCD1F000ECD2368
:106CA00004D000EBCCF101EBCDF1CCC1F3FFCDC1B1
:106CB000F4FF41E9E7CFD9FF1200D2D886E949E8CD
:106CC000C9D800EBE6FF01EBE6FF13EC38F044E92E
:106CD000C1D8A6EC34F042E9F3500E6E0E50025CBF
:106CE0000E6E0E3401E30E6A0E50025C0101CC6F91
:106CF000CD6B800B01E0CD69CCC1E6FFCDC1E6FFD5
:106D0000A9D80EEBD0F1D16BD0BFD1690350D025FB
:106D1000CE6F0450D121CF6FCEC1E6FFE66ED1EC2D
:106D200033F046E94AE9E7CFD9FF120099D886E95E
:106D3000013402E32D0E01D02B0EE66E03EBE9FFCA
:106D400004EBEAFFE552E750EF6E00EBE6FF01EBE4
:106D5000E6FF99DF42E9F3CFE6FFF4CFE6FF02EB6F
:106D6000E6FF03EBE6FF04EBE6FFA7DF45E941E9B9
:106D7000E7CFD9FF120074D887E941E8076A0334E6
:106D80000350071802E60350075C36E203EBD0F12C
:106D90000101D16BD0BFD1693FD8D2BFD36965D8CB
:106DA000EF380F0BF66EF76AF6BEF76849D8CC6F6E
:106DB000CD6B800B01E0CD693CD8E552E750EF6E1A
:106DC00003EBD0F1D16BD0BFD16926D8D2BFD36944
:106DD0004CD8EF500F0BF66EF76AF6BEF76830D856
:106DE000010FCC6FCD6B800B01E0CD6922D8E5524D
:106DF000E750EF6E072AC3D700500AE00750E82497
:106E00000101CC6FCD6B800B01E0CD6912D8EF6A28
:106E100042E9E7CFD9FF12000150D025CE6F0250D2
:106E2000D121CF6FCE07000ECF5B07EBD2F1D36B32
:106E30001200CC510424E96ECD510520EA6E1200F7
:106E4000AC0EF6267D0EF7220800F550E66E0750D0
:106E5000E8241200D950060FE66EDACFE6FF1200E2
:106E6000D9CFE6FFE1CFD9FF1200D251CE5DE96E56
:086E7000CF51D355EA6E120068
:086E780081B804D06DB604D00E
:106E80000FD802D06DB613D80201A60508E16DBA7D
:106E900006D0686A696A69806988020EA66F120066
:106EA0006D6A696A6D860201010EA66F12006D6A35
:106EB000696A0201A66B120057EF37F00201A65172
:106EC00001E112006850040B04E06950040B01E07A
:106ED00045D86DB212006850010B04E06950010BF7
:106EE00001E069D86850100B04E06950100B01E014
:106EF0002ED86850400B04E06950400B01E047D8A1
:106F00006850200B04E06950200B01E042D8685023
:106F1000020B04E06950020B01E04BD8030E0201A2
:106F2000A65D01E212000201AE6B040EAE5D0EE240
:106F30006850080B0BE06950080B08E0ABEC2FF031
:106F4000000901E168960201AE2BEFD712006984B7
:106F500068986D82A19AA08AA09A12006D92699495
:106F600068A402D06894FCD712000201A7A10ED039
:106F70006D926D840201080EAF6F070EB06FAF0700
:106F8000000EB05BAF51B011FAE16D941200689C35
:106F9000120070A00CD0800E0401005D07E1840E89
:106FA0000401045D03E104018C0E006F7090689A87
:106FB00012006A6A12006A6A686A9F0E6B6E7B0E24
:106FC000696E6E6A0F0EE66E710EE66E0F0EE66E5D
:106FD00018D843E9160E706E68A608D068960000AF
:106FE00000000000000000000000F6D76D98C2EC21
:106FF00030F00201A7910201A86B0201030EA66FF7
:107000001200D9CFE6FFE1CFD9FF84E901EBE9FF18
:1070100002EBEAFF005003E0EE6A0006FBD741E90D
:06702000E7CFD9FF1200CA
:0A702600D9CFE6FFDACFE6FFFA0E3D
:10703000E3CFD9FFFB0EE3CFDAFFFD0EE35209E702
:107040002D0EDE6EFC0EE31EE32AFD0ED8B4E30621
:10705000E31EE652E652E652FD0EE124E76EFF0E15
:10706000E220E46EE652F70EE3CFE6FFF70EE3CF41
:10707000E6FF83EC38F0F90EE124E96EFF0EE22022
:10708000EA6E73EC38F00AE170EC38F009E173EC69
:1070900038F008E170EC38F007E108D07EEC38F009
:1070A00079EC38F07EEC38F079EC38F07EEC38F0A2
:1070B000DE6AF90EE126FF0EE222FF0EE3CFDAFFD1
:1070C000E552FF0EE3CFD9FFE552FC0EE124E96E55
:1070D000FF0EE220EA6EEECFF3FFEFCFF4FF1200D7
:1070E000EF380F0B1200EF500F0B02E1EE52D88475
:1070F0001200EF380F0B300FDE6E1200EE500F0B48
:10710000300FDE6E1200FC0EE3CFE9FFFD0EE3CF81
:10711000EAFF100EE66EEE6AEE6AEF6AD890FD0E98
:10712000E336FE0EE336ED36ED36EF36FF0EE306C0
:1071300009E0A4EC38F0EE52A4EC38F0EE52A4ECE6
:1071400038F0EDD7E56E1200030EEF24E8B6EF6ECF
:0A715000300EEF24E8BEEF6E000CD5
:06715A000000000000002F
:107160005F00000000030003000006090906242A4E
:107170007F2A1223130864623649562050000B07F9
:10718000000000003E410000413E0000082A1C2A89
:107190000808083E080800583800000808080808D1
:1071A000003030000020100804023E5149453E00E6
:1071B000427F4000625149494622414949361814EC
:1071C000127F1027454545393C4A4949300171092C
:1071D00005033649494936064949291E0036360015
:1071E00000005B3B00000008142241141414141426
:1071F000412214080002015109063E415D551E7EE0
:107200000909097E7E494949363E414141227F4173
:1072100041413E7F494949417F090909013E4141B8
:1072200051327F0808087F00417F410020404040E4
:107230003F7F081422417F404040407F020C027F84
:107240007F0408107F3E4141413E7F090909063E07
:107250004151215E7F0919294626494949320101D8
:107260007F01013F4040403F07186018077F20180A
:10727000207F6314081463030478040361514945B3
:0172800043CA
:0F7281003030303020303030300030303033009B
:1072900030303020303030005858585858585858EE
:1072A00020585858585858585820585858585858CE
:1072B00058580048697961004552585800434C5865
:1072C00058004C303030004D30303000484F4C4486
:1072D0000053415645005241572000484947480055
:1072E000475241440043414C20002030302300539A
:1072F00041502000303030250048454C500030309F
:1073000030300030303047004330303000303030E3
:1073100023002A20200D0A0024505450534854447E
:107320002C003030303030300041545A0A00415483
:107330002B42545343414E2C332C300A0041542BE2
:1073400042544D4F44452C330A0041542B42544E75
:10735000414D453D22536865746C616E64204174F3
:107360007461636B20506F6E79222F6E0041545A06
:037370002F6E007D
:0D7373001201000202000020D8040A0000F0
:1073800000010200010902430002010080320904E9
:107390000000010202010005240010010424020281
:1073A00005240600010524010001070582030800E9
:1073B0000209040100020A00000007050302400060
:1073C000000705830240000004030904340355004C
:1073D0006E0064006500720077006F006F0064004B
:1073E000200055006E0064006500720067007200A6
:1073F0006F0075006E006400200020002000200057
:10740000340353006800650074006C0061006E0076
:1074100064002000410074007400610063006B0090
:10742000200050006F006E00790020002000200036
:107430002000200085738573C873CC730074586274
:107440002A0EF66E080EF76E000EF86E02010900A5
:10745000F5508F6F0900F550906F03E18F6701D0F1
:107460003DD00900F5508A6F0900F5508B6F090077
:10747000F5508C6F09000900F550E96E0900F550D0
:10748000EA6E090009000900F5508D6F0900F550FA
:107490008E6F09000900F6CF91F2F7CF92F2F8CF84
:1074A00093F28AC2F6FF8BC2F7FF8CC2F8FF02018B
:1074B0008D5302E18E5307E00900F550EE6E8D0703
:1074C000F8E28E07F9D791C2F6FF92C2F7FF93C296
:0E74D000F8FF02018F07000E905BBFD712007D
:0274DE00D9CF04
:1074E000E6FFDACFE6FFE1CFD9FFE2CFDAFF87E9A7
:1074F000E6EC3EF0C580C5B0FED7A1B62CD004EBBB
:10750000E6FF35D80FE1C5BC28D003EBE6FF2FD846
:1075100009E1C5BC22D0C582C5B2FED70428E66EFB
:1075200026D803E0C584FD0E1CD0C5BC16D000EBE8
:10753000E6FF01EBE6FF02EBE6FFA3EC3CF043E9DC
:10754000000909E1C58AC588C5B8FED7C584C5B498
:10755000FED7A1A605D0FF0E04D0C584FE0E01D033
:10756000000E41E9E5CFDAFFE7CFD9FF1200F7ECD3
:087570003CF041E900091200A2
:08757800D9CFE6FFDACFE6FFF0
:10758000E1CFD9FFE2CFDAFF84E9E6EC3EF0C58037
:10759000C5B0FED7A1B626D001EBE6FF33D811E186
:1075A000C5BC22D000EBE6FF2DD80BE1C5BC1CD03A
:1075B000C582C5B2FED7A1B615D00128E66E22D885
:1075C00003E0C584FD0E12D0C5BC0ED0C586C5B67D
:1075D000FED7C58AC588C5B8FED7C584C5B4FED751
:1075E000A1A607D0F36803D0C584FE0EF36EF4683D
:1075F00003D0C950F36EF46A41E9E5CFDAFFE7CF73
:0E760000D9FF1200F7EC3CF041E9000912003E
:02760E00D9CFD2
:10761000E6FFDACFE6FFE1CFD9FFE2CFDAFF85E977
:10762000AC6AAB6A02B0AC8802A202D0AC8CAB8C64
:1076300002B4AC8E02A602D0AB8801D0AB8A02B8ED
:10764000AC849E9802BAAB8602AC02D09D8A01D06F
:107650009D9A9E9A02AE02D09D8801D09D9800EB23
:10766000AFFF010101EBCCF1CD6BCCC1B0FFAC8A17
:10767000AB8E949C948EAC50100B04E0AC50800BFD
:1076800001E1948C41E9E5CFDAFFE7CFD9FF1200A1
:10769000D9CFE6FFDACFE6FFE1CFD9FFE2CFDAFFBD
:1076A00085E9E6EC3EF0C580C5B0FED7A1B61BD09B
:1076B00002EBE6FF21D80CE1C5BC0DD001EBE6FFE3
:1076C0001BD806E1C5BC07D000EBE6FF15D806E0E5
:1076D000C584FD0E0BD0C584FE0E08D0C584C5B48C
:1076E000FED7A1A602D0FF0E01D0000E41E9E5CFE2
:1076F000DAFFE7CFD9FF1200F7EC3CF041E90009CF
:02770000120075
:0E770200000000000000000000000000000079
:107710000000000000000000000000000000000069
:107720000000000000000000000000000000000059
:107730000000000000000000000000000000000049
:107740000000000000000000000000000000000039
:107750000000000000000000000000000000000029
:0A776000000000000000000000001F
:06776A00F36AF46AFF0E51
:10777000E124E96EFF0EE220EA6EED6613D02F0ED3
:10778000EF6410D0390EEF640CD0400EEF640AD0D5
:107790005A0EEF6406D0600EEF6404D07B0EEF60EB
:1077A00001D0F32A1200F36AF46AFF0EE124E96EB5
:1077B000FF0EE220EA6EED660AD0200EEF5C06E0D6
:1077C000080EEF6404D00E0EEF6001D0F32A120011
:1077D000D9CFE6FFE1CFD9FF82E941E8080E026E7A
:1077E00000EBB2F28B940201B2BF8B840000000068
:1077F000D8908BB4D8808B90B23700000000000086
:107800000000000000000000000000000000000078
:107810008B808B940201B2BF8B8402060250E8E198
:0E7820000201B25100D042E9E7CFD9FF1200B9
:02782E00D9CFB0
:10783000E6FFDACFE6FFE1CFD9FFE2CFDAFF83E957
:1078400044E8F8CF05F0F6CF06F00C0EBA6E050E40
:10785000F66EF76A300EF86E0800F550010B02E084
:10786000046801D0046A045002E0949201D0939617
:10787000CA9400EBCBFFCA8405C0F8FF06C0F6FF30
:0C78800045E9E5CFDAFFE7CFD9FF1200A1
:04788C00D9CFE6FF6B
:10789000DACFE6FFE1CFD9FFE2CFDAFF85E9C26AAE
:1078A000C06A01407F0B3C0BC26E0138F00B300BFD
:1078B0000010C16E0250040DF350380B0101CD6F62
:1078C00002380F0B070BCC6F800E0214CC11CD11B8
:1078D000C06E01AE03D09E9C9D8CF28CC28041E9AB
:0A78E000E5CFDAFFE7CFD9FF120071
:0678EA00D9CFE6FFDACF62
:1078F000E6FFE1CFD9FFE2CFDAFF85E9ACA2FED700
:1079000000EBF6FF01EBF7FF02EBF8FF0800F5CF05
:10791000E6FF7AEC3EF041E9D9CFE9FFDACFEAFFA2
:10792000EFCFF6FFEE2AEFCFF7FF000EEE22EFCFFC
:10793000F8FFEE220800F550E1E141E9E5CFDAFF7A
:06794000E7CFD9FF1200A1
:0A794600D9CFE6FFDACFE6FFE1CF6C
:10795000D9FFE2CFDAFF85E90050000600091AE0FE
:10796000F9EC3EF0E66E01EBE9FF02EBEAFF012ADB
:10797000000E0222E552E750EF6EC5B6FED7A1A673
:1079800002D0FF0E08D00050E7E0C59AC588C5A810
:10799000E3D7FDD7000E41E9E5CFDAFFE7CFD9FF06
:0279A0001200D3
:0E79A200D9CFE6FFDACFE6FFE1CFD9FFE2CF83
:1079B000DAFF84E942E880EB04F081EB05F0060E83
:1079C000D89004360536E804FBE105EBBBFF044024
:1079D000E8423F0B300B0101CC6FCF0EBA14CC1133
:0E79E000BA6E43E9E5CFDAFFE7CFD9FF120018
:0279EE00D9CFEF
:1079F000E6FFDACFE6FFE1CFD9FFE2CFDAFF83E996
:107A000000EBC9FFC6AE02D0FF0E11D0C7B0FED743
:107A10000F0EC614080804E00F0EC614090802E190
:107A2000E6EC3EF0C5AC02D0FE0E01D0000E41E9FE
:0A7A3000E5CFDAFFE7CFD9FF12001F
:067A3A00D9CFE6FFDACF10
:107A4000E6FFE1CFD9FFE2CFDAFF84E9ACA2FED7AF
:107A500000EBE9FF01EBEAFFEFCFE6FF7AEC3EF047
:107A600041E900EBE9FF01EBEAFF002A000E0122E9
:107A7000EF50ECE141E9E5CFDAFFE7CFD9FF1200A3
:107A8000D9CFE6FFDACFE6FFE1CFD9FFE2CFDAFFC9
:107A900083E9360E0014B16EB36AB26AA19200AEE9
:107AA00002D0A08201D0A09200A002D0B18E01D05D
:107AB000B19EB18041E9E5CFDAFFE7CFD9FF1200EF
:107AC000D9CFE6FFDACFE6FFE1CFD9FFE2CFDAFF89
:107AD00083E97E0E0014CD6E00AC02D0CD8E01D0B5
:107AE000CD9ECF6ACE6A9E9000AE02D09D8001D01E
:107AF0009D90CD8041E9E5CFDAFFE7CFD9FF1200B5
:107B0000FF0EE3500201B16FEE0E02D0F20E000044
:107B1000E76EE72E89EF3DF00C0E0101FF6FE76A7B
:107B2000E72E90EF3DF0FF2F8FEF3DF00201B12FD8
:067B300086EF3DF012009B
:0A7B3600D9CFE6FFDACFE6FFE1CF7A
:107B4000D9FFE2CFDAFF83E97F0E0014D56ED76A42
:107B5000D66AF29400AE02D0F28A01D0F29AD58EA3
:0C7B600041E9E5CFDAFFE7CFD9FF1200C2
:047B6C00D9CFE6FF88
:107B7000DACFE6FFE1CFD9FFE2CFDAFF83E9FB0EF0
:107B80000014CA6ECC6A9E9200AE02D09D8201D0D3
:107B90009D92CA8441E9E5CFDAFFE7CFD9FF120011
:107BA000D9CFE6FFDACFE6FFE1CFD9FFE2CFDAFFA8
:107BB00084E93F0EC716C66AC56A0150C612005056
:107BC000C71293829380C68A41E9E5CFDAFFE7CFF7
:047BD000D9FF1200C7
:0C7BD400D9CFE6FFDACFE6FFE1CFD9FF02
:107BE000E2CFDAFF84E942E880EB04F081EB05F0B4
:107BF00005EBB3FF04EBB2FF43E9E5CFDAFFE7CFD4
:047C0000D9FF120096
:0C7C0400D9CFE6FFDACFE6FFE1CFD9FFD1
:107C1000E2CFDAFF82E942E8B250026EB350036E5F
:107C200002EBF3FF03EBF4FF43E9E5CFDAFFE7CF25
:047C3000D9FF120066
:0C7C3400D9CFE6FFDACFE6FFE1CFD9FFA1
:107C4000E2CFDAFF84E942E880EB04F081EB05F053
:107C500005EBCFFF04EBCEFF43E9E5CFDAFFE7CF3B
:047C6000D9FF120036
:0C7C6400D9CFE6FFDACFE6FFE1CFD9FF71
:107C7000E2CFDAFF82E942E8CE50026ECF50036EC7
:107C800002EBF3FF03EBF4FF43E9E5CFDAFFE7CFC5
:047C9000D9FF120006
:0C7C9400D9CFE6FFDACFE6FFE1CFD9FF41
:107CA000E2CFDAFF84E942E880EB04F081EB05F0F3
:107CB00005EBD7FF04EBD6FF43E9E5CFDAFFE7CFCB
:047CC000D9FF1200D6
:0C7CC400D9CFE6FFDACFE6FFE1CFD9FF11
:107CD000E2CFDAFF82E942E8D650026ED750036E57
:107CE00002EBF3FF03EBF4FF43E9E5CFDAFFE7CF65
:047CF000D9FF1200A6
:0C7CF400D9CFE6FFDACFE6FFE1CFD9FFE1
:107D0000E2CFDAFF83E9ACAC04D0AC900201B3B3AC
:107D1000AC8000EBADFF41E9E5CFDAFFE7CFD9FF5B
:027D200012004F
:0E7D2200D9CFE6FFDACFE6FFE1CFD9FFE2CFFF
:107D3000DAFF83E900EBB8FF41E9E5CFDAFFE7CFEF
:047D4000D9FF120055
:0C7D4400FF0EE3500201B16F1A0E00D0D8
:107D500000D001D0200EE76EE72EFED7B12FFAD764
:047D600000D012003D
:0C7D640013EE00F023EE00F0F86A20ECB3
:0E7D70003AF011EC3FF0CFEC04F0FBD712001C
:027D7E00C4CF70
:107D8000CEF1CEC1CFF10101CE6BC350CE11F36E57
:067D9000CFC1F4FF120058
:0A7D9600FF0EE350E84E120000005B
:0C7DA00000D000D000D0E82EFAD712006E
:047DAC00303132330D
:0D7DB00034353637383941424344454600EA
:017DBD0000C5
:027DBE00898AB0
:0C7DC0008B948B80929A94949490120003
:047DCC001F0EC514AD
:0A7DD000FDE1C750040BFAE11200B8
:067DDA0000EE00F00F0EA8
:087DE000EE6AEA62FDD7120011
:087DE8000A4F4B0A000A4B4F41
:027DF0000A0087
:0A7DF200C586C7A0FED7C9501200D5
:047DFC00C250020B64
:067E000001E0010E12007A
:067E0600B190A0921200F1
:047E0C00C2909D9CE7
:027E100012005E
:047E1200898A120047
:047E1600C69A1200F6
:047E1A00899A12002F
:027E1E00C2821E
:027E200012004E
:027E220012004C
:047E24003D0A2700EC
:087E2800C7711C010000000AF3
:057E300000000100004C
:067E350001FFFFFFFF0149
:017E3B000343
:047E3C00B84B390006
:087E400049920400000040001B
:020000040030CA
:0100000038C7
:010001000EF0
:010002001CE1
:010003001CE0
:01000500807A
:01000600C138
:010008000FE8
:01000900C036
:01000A000FE6
:01000B00E014
:01000C000FE4
:01000D0040B2
:0200000400F00A
:0100FF00AA56
:00000001FF
